:040000000C94BA01A1
:080024000C94AA020C9479026D
:040040000C940D050A
:040048000C9475217E
:040078000C94551877
:14008C00D723DC23E123E623EB23F023F523FA23FF230424BA
:1400A00009240E24132418241D24222427242C2431243624A9
:1400B4003B24402445244A242E254F245D25622567256C25B2
:1400C800712576257B25802585258A258F25942599259E2567
:1400DC00A325A8256326AD25922697269C26A126A626AB2685
:1400F000B026B526BA26BF26C426C926CE26D326D826DD26BF
:140104004A27E226E62DEE2DF62DFE2D062E0E2E162E1E2EF2
:14011800262E2E2E362E3E2E462E4E2E562E5E2E662E6E2E23
:14012C00762E7E2E822E862E8A2E8E2E922EE82EEC2EF42E85
:14014000FC2E042F0C2F112F162F1B2F202F282F302F382FD8
:14015400402F482F502F542FBF30C430C930CE30DB30E030BA
:14016800E530EA30EF30F430F930FE30033108310D311231CC
:14017C0017311C3127314331553159315D316D318131863169
:140190008A3178348F34A734BE34D134E534993599353E3537
:1401A400423599359935993599359935993599359935993592
:1401B80099356A356E35823566350C3599356235F8345A3570
:1401CC00993502355635993599359935993599355E3524478B
:1401E00050524D432C00000302050003050104060204010089
:1401F4000100D00700000000000000001F003B005A007800F3
:140208009700B500D400F300110130014E016D0100FFFFFFD2
:14021C00FFFF000020203F0020204A5441470020205761747F
:140230006368646F6700202042726F776E2D6F7574002020A8
:1402440045787465726E616C002020506F776572204F4E0059
:1402580020200052657365742044617465202F2054696D65B3
:14026C00202020202020205265736574205479706500436F27
:140280006D6D756E69636174696F6E20746F20475053206435
:140294006576696365206661696C656400453300436F7272B7
:1402A800656374656420746F206C6F63616C2074696D653A06
:1402BC0020200054696D653A2020004461746520284D2F445F
:1402D0002F59293A2020005554432028477265656E77696387
:1402E40068292044617465202F2054696D653A00285365655A
:1402F8002048656C7020666F722073746174757320636F64C8
:14030C006573290047505320436F6D6D756E69636174696FEA
:140320006E205374617475733A20004D4355435352005275C9
:140334006E6E696E6700562B204C4F5700562B204F4B004984
:140348004E4954003031323334353637383961626364656654
:14035C006768696A6B6C6D6E6F707172737475767778797AC3
:0303700000010089
:14037400CFEFD0E1CDBFDEBFC051D0400AEA08830024EBE747
:14038800F2E014E0E03FF10711F00192FBCF0083E8EFF1E0FB
:14039C00A0E0B1E013E0E337F10721F0C89531960D92F9CF9B
:1403B0000E94230AFFCF0E94C23D002321F4599A83E089B92B
:1403C40011C0013021F4599885E089B90BC0023021F4599873
:1403D80087E089B905C0033019F4599887E189B986E080934F
:1403EC00950088E98AB9ACB078940E94B03D08952CB0209292
:140400007B0208955D9BFECF0CB908950E94C53D6801AA24CC
:14041400BB240AC0F60100810E94833EC50101965C01C601CF
:1404280001966C01F6012080222091F7A89501E010E00E94AB
:14043C00BC3D089508950E94C23D87B1806C87B927B027B8BE
:14045000329A379A85B7806185BF85B7806485BF88950027F2
:1404640022D05801379885B78F7B85BF0E94B03D089587B17C
:14047800806C87B927B0202A27B886B1856086B9379A08957B
:14048C0037980895379A369A089504B1112725B03324322C3B
:1404A0002224020D131D349A08950E94C23D379A27B0202AC5
:1404B40027B8369A3699FECFA4B0BB2425B03324322C2224E6
:1404C800A20CB31C85010E94B03D0895222425BC87B78F738A
:1404DC0087BF8DE484BD83EB83BD87B7806487BF85E085BD57
:1404F00008958A939A938FB78A938DE484BD809181028F5F7A
:1405040080938102809180028F5F8093800280917F028F5FB7
:1405180080937F0280917E028F5F80937E0289918FBF999197
:14052C0089911895222425BC87B78F7387BF88E384BD88EC27
:1405400083BD87B7806887BF8CE085BD0895222424BC0895ED
:140554008A939A938FB78A9380917E028F5F80937E028091C3
:1405680081028F5F8093810289918FBF999189911895889AFD
:14057C00899A909A919A0895909A919A899A91980895899AF5
:1405900091989098909A919A0895909A0000909808950E9483
:1405A400C53DC02E899A9098AA240BC08C2D8078803811F401
:1405B800919A01C09198909ACC0C9098A3948A2D883090F3C7
:1405CC001CD00023E9F70E94BC3D08950E94C53DCC24AA2492
:1405E0000AC0CC0C8998909A819B03C08C2D8160C82E909883
:1405F400A3948A2D883098F3CEDF0C2D0E94BC3D089500277D
:1406080090988998909A819B01C001E0909808950E94C53D44
:14061C00A22EC02E90988C2D8870883011F4919A01C0919861
:14063000B4DF8C2D8470843011F4919A01C09198ACDF8C2D64
:140644008270823011F4919A01C09198A4DF8C2D8170813006
:1406580011F4919A01C091989CDF8A2D8470843011F4919A6A
:14066C0001C0919894DF8A2D8270823011F4919A01C09198A8
:140680008CDF8A2D8170813011F4919A01C0919884DF0C8099
:14069400002011F0919A01C091987DDFB2DF0023E9F70E948A
:1406A800BC3D08950E94C93DA22EE02E2197CF80D88464DF7C
:1406BC00222428822E2D0AE0A9DF0A2D6CDF00276ADF80E01B
:1406D00091E05C0107C0F60101916F0162DFC50101975C018C
:1406E400AA20B9F7BB20A9F750DF21960E94BF3D08950E944A
:1406F800C53D5901C02E219741DF222428822C2D0AE086DF34
:14070C008501012F112747DF0A2D107044DF0D8142DF37DF26
:1407200021960E94BC3D08950E94C53D6901A02E219728DF3B
:14073400222428822A2D0AE06DDF8601012F11272EDF0C2DFF
:1407480010702BDF1BDF81E088832A2D0AE060DF3FDFA02E41
:14075C0018DF0A2D21960E94BC3D08950027112702C00F5FDD
:140770001F4F0037E7E11E07D0F308950E94C53DA02EA895D4
:14078400C0900401DD24CC2011F4DD20B9F0C6018130E0E03C
:140798009E0709F430C08230E0E09E0709F44DC08030E0E02A
:1407AC009E070CF47EC0C6018930E0E09E0709F456C077C027
:1407C0008EED91E0E0910301FF27E80FF91FE491AE1631F431
:1407D400809103018F5F8093030103C0222420920301809127
:1407E8000301873009F0F8C081E0809304012224209205011A
:1407FC00F1C08A2D8C3289F48CE992E0E0910501FF27E80FCB
:14081000F91F2224208220920501809104018F5F8093040100
:14082400DDC08CE992E0E0910501FF27E80FF91FA08280915D
:1408380005018F5F80930501CFC08A2D8C3249F42224209266
:14084C000501809104018F5F80930401C3C0A092940280911A
:1408600005018F5F80930501BBC08A2D8C3289F485E992E02A
:14087400E0910501FF27E80FF91F2224208220920501809113
:1408880004018F5F80930401A7C085E992E0E0910501FF276D
:14089C00E80FF91FA082809105018F5F8093050199C08A2DE9
:1408B0008C3229F4809104018F5F809304018A2D8A3009F0D3
:1408C4008DC022242092040120920301AA243DC02A2C3324A8
:1408D800220C331C8CE992E0F101E80FF91F40808AE0849D5C
:1408EC00C001805E9140EDE9F2E0D101AE0FBF1F9C91905363
:14090000890FE1E9F2E0AA2DBB27AE0FBF1F8C932A2C33248F
:14091400220C331C85E992E0F101E80FF91F40808AE0849D26
:14092800C001805E9140E6E9F2E0D101AE0FBF1F9C9190532D
:14093C00890FEEE8F2E0AA2DBB27AE0FBF1F8C93A3948A2D06
:14095000833008F4BFCF82E892E0E8E8F2E006E010E0FA9375
:14096400EA939A938A930E946B3E2090910220928202209044
:14097800920220928302209093022092840220908E02209231
:14098C00850220908F022092860220909002209287021CE3D9
:1409A00000918A020F5F0E94583D20908402201631F48091DF
:1409B40001018F5F8093010105C022242092010120920201B6
:1409C80080910101843041F481E080930201809101018150C4
:1409DC00809301010E94BC3D0895F89483B78F7B83BF83B76E
:1409F000877F83BF83B78D7F83BF83B7856083BF87B78C7F79
:140A040087BF80B7886080BF222422BE87B7816087BF7894A3
:140A180008952A928A939A932FB62A9280912A0390912B03F9
:140A2C00019690932B0380932A038091AC028F5F8093AC0220
:140A400081E080937B03809367038091F0048F5F282E209238
:140A5400F0048BE3821530F422242092F00481E08093AB0264
:140A680029902FBE99918991299018958091F1048F5F282EE0
:140A7C002092F1048C3309F0CCC022242092F10481E080931A
:140A90007A038091F2048F5F282E2092F204883109F062C00E
:140AA40022242092F2042092A30281E08093AA028091F304D1
:140AB8008F5F282E2092F304803249F48091F4048F5F809344
:140ACC00F40481E08093F30439C08091F3048F3199F4809154
:140AE000F404843031F0863021F0893011F08B3059F580919A
:140AF400F4048F5F8093F40481E08093F30422C08091F304A8
:140B08008E3159F48091F4048230D1F48F5F8093F40481E0F3
:140B1C008093F30413C08091F3048D3179F48091F4048230FA
:140B300059F476D0002341F08091F4048F5F8093F40481E067
:140B44008093F3048091F4048D3041F481E08093F40480911B
:140B5800F5048F5F8093F50476D00093F6045BC08091F204A1
:140B6C00853089F480E19EE090932D0380932C032224332432
:140B800030922B0320922A032090E1032092A90246C080918A
:140B9400F204823009F041C08091F4048330D9F487E020900B
:140BA800F3048215B0F4822D8F3098F48091F604813079F4E4
:140BBC0081E08093A8022FE130E000270E949403013029F439
:140BD0008091F2048F5F8093F2048091F4048B30F1F4809159
:140BE400F3048830D0F48091F6048130B1F422242092A80287
:140BF8002FE130E000270E949403002361F02090A30222205E
:140C0C0041F48091F20481508093F20481E08093A302089508
:140C200014E60091F5040E94583D002341F420E931E0009102
:140C3400F50411270E94AD3C07C024E030E00091F504112753
:140C48000E94AD3C08950E94C53D2C9786EE91E0FE010CE039
:140C5C0010E0FA93EA939A938A930E94523E8091F504992744
:140C70008053984F9093A6028093A5028091F5049927805394
:140C8400984F5C018091F404833020F481E090E06C0102C048
:140C9800CC24DD24AC18BD0824E030E085010E94B13C15018F
:140CAC00200E311E24E630E085010E94B13C201A310A20E90A
:140CC00031E085010E94B13C200E311ECE010197E091F404AD
:140CD400FF27E80FF91F40805524240C351C4090F3045524DD
:140CE800240C351C27E030E081010E94AD3C0F5F1F4F2C96B5
:140CFC000E94BC3D08952FE130E000270E949403002309F40C
:140D100062C09DDF0093F6042FE130E000270E949403002301
:140D240009F454C08091F404833009F58091F304883020F41C
:140D380022242092A80248C087E02090F304821580F4822D35
:140D4C008F3068F487502090F604821520F081E08093A80232
:140D600037C022242092A80233C081E08093A8022FC083E083
:140D74002090F404821538F4822D8B3020F481E08093A80264
:140D880023C08091F4048B30A1F48091F304883060F4309047
:140D9C00F604831520F022242092A80213C081E08093A8020E
:140DB0000FC022242092A8020BC08AE02090F404821518F042
:140DC400822D843018F422242092A8020091A80201C00027E7
:140DD80008950E94C93DAA24BB24C801805D974083709070A5
:140DEC008030890721F481E090E06C0102C0CC24DD24EC2C95
:140E000016C0C801805D9740837090708030890721F481E0E2
:140E140090E06C0102C0CC24DD2420901E0130901F012C0C53
:140E28003D1CA20CB31C18010150104080ED97E08215930513
:140E3C0010F382E0821730F4EE2021F081E090E06C0102C061
:140E5000CC24DD2482E0829FF00184E091E0E80FF91F2080A5
:140E640031802C0C3D1CA20CB31C2E803324A20CB31C8501B3
:140E78000E94BF3D08953A932A930E94C93D3801269782EF92
:140E8C0091E0FE0106E010E0FA93EA939A938A930E94523E86
:140EA0008EE691E04C01EE24E394AA2422C00C841D84081882
:140EB40019081D860C868C819D8101969D838C83805D97402F
:140EC800837090708030890721F481E090E06C0102C0CC24DE
:140EDC00DD24EC2C2E2C332440901E0150901F01420C531C8C
:140EF00042010C841D8480149104C8F28CE0A82E3DC082E0F6
:140F04008A1530F4EE2021F081E090E06C0102C0CC24DD2406
:140F180082E08A9DF00184E091E0E80FF91F208031802C0CDE
:140F2C003D1C0C841D842014310408F582E08A1530F4EE208E
:140F400021F081E090E06C0102C0CC24DD2482E08A9DF00121
:140F540084E091E0E80FF91F208031802C0C3D1C0C841D8492
:140F6800021813081D860C862A2C33243B822A8205C0AA94F2
:140F7C0022242A1408F4BFCF0C841D8419820882CE0106E048
:140F900010E07A926A929A938A930E946B3E26960E94BF3D66
:140FA40022960895222420929A0020929B0086E080939D00EF
:140FB8008FEB809399002092980088E980939A0008952224B4
:140FCC0020929A00089588E980939A00089500919C000895A3
:140FE000222420929A0020929B0086E080939D008FEB80937B
:140FF40099002092980088E980939A000895222420929A00B9
:14100800089588E980939A00089500919C0008950E94C93D0A
:14101C00C22E58012997222433243092B4022092B302A895FE
:1410300024E039E000270E949403202E3324322C22243C8228
:141044002B8225E039E000270E949403202E33240B801C80A1
:14105800020C131C1C820B820F8408822C2D85010E94ED068B
:14106C001E830D8320E039E000270E949403202E3324388663
:141080002F8221E039E000270E949403A02EBB2422E039E069
:1410940000270E949403E02ECE2CDD24DC2CCC2423E039E0CB
:1410A80000270E949403E02E2E2C3324C20CD31C2F803884ED
:1410BC0028822A2D86010E94ED0668012D803E80201A310ABA
:1410D0003A8229822B813C8181013AD129960E94BF3D0895B5
:1410E4000E94C53DC02E2090F2048CE3829D50012090F1043C
:1410F8003324A20CB31CA895CC2009F46DC022243092B402FF
:14110C002092B302910104E010E00E94703DF80184ED92E0D7
:14112000E80FF91F208031802A143B0408F058C036C0209127
:14113400B3023091B40204E010E00E94703D84ED92E0F8017C
:14114800E80FF91F2080318088ED92E0F801E80FF91F408084
:14115C0051804214530408F425C02091B3023091B40204E05F
:1411700010E00E94703DF80188ED92E0E80FF91F20803180EC
:14118400A214B30408F412C08091B3029091B40201969093C5
:14119800B4028093B3028091B3029091B4028F30E0E09E0704
:1411AC000CF4C1CF2091B3023091B40204E010E00E94703D9F
:1411C000F80186ED92E0E80FF91F00813BD08091B3029091BB
:1411D400B40201969093B4028093B3028091B3029091B4027C
:1411E8008031E0E09E073CF59C0104E010E00E94703DF801F3
:1411FC0084ED92E0E80FF91F20803180A214B304C1F42091C9
:14121000B3023091B40204E010E00E94703DF80186ED92E09D
:14122400E80FF91F00810CD08091B3029091B40201969093F3
:14123800B4028093B3020E94BC3D08950E94C23DA02E80E31A
:14124C008A9DC001885E9E4F5C01A8959C0100270E9494033C
:141260000093AE0395012F5F3F4F00270E9494030093AD03E1
:1412740095012D5F3F4F00270E9494030093CE03202E87E637
:14128800829D800100571E4F24E630E00E94B13C0093CD03E2
:14129C002090CE038EE6829D800106571D4F24E630E00E9424
:1412B000B13C0093CC0395012C5F3F4F00270E949403009339
:1412C400640395012B5F3F4F00270E9494030093D60395019F
:1412D8002A5F3F4F00270E9494030093AC039501295F3F4F9D
:1412EC0000270E9494030093AB039501285F3F4F00270E94D9
:1413000094030093AF039501265F3F4F00270E949403009361
:141314006F0381E0809335038091E203813011F0833069F4EF
:141328002090AE03222021F42090AF03222029F01A9A81E027
:14133C008093340304C01A982224209234030E94B03D089582
:141350000E94C93D590168012297A895C6018030E0E09E074C
:141364003CF0A816B90624F0AA2081F4BB2071F48091F6042E
:1413780099278C5F964F5C018091F604813041F4C501079620
:14138C005C0104C0C601835F964F5C01950100270E9494034B
:1413A000A02E80E58A9DC001885E9B4F99838883CC24DD2436
:1413B4003EC003E010E096010E94703DE880F980E00EF11E90
:1413C800970100270E949403A02EBB24BA2CAA2497012F5F92
:1413DC003F4F00270E949403202E3324A20CB31C04E010E019
:1413F00096010E94703DF80184ED92E0E80FF91FB182A082C3
:1414040097012E5F3F4F00270E949403202E04E010E0960108
:141418000E94703DF80186ED92E0E80FF91F332431822082D8
:14142C00C60101966C018FE090E08C159D0508F0BCCF229684
:141440000E94BF3D089521978BEE81BB00E40E94313C00E419
:141454000E94313C00E40E94313CF89484B7806884BF84B755
:14146800806884BF66270E94F30405E00E943B02789400EA65
:14147C0016E821E030E00E94493C05E00E9455028BE992E062
:141490008017910734F422242092A7030E94072012C000EACA
:1414A40016E821E030E00E94493C81E0809378030E94C0208D
:1414B80080916200877F809362000E94E120F8940E946A02F5
:1414CC000E9444210E94BD0278940E94D31606991CC1C19A36
:1414E00081E08093AE03199886B3827086958093A5032224DB
:1414F400332430922B0320922A037EC0A895209081022220CE
:14150800A1F020908303222039F000E20E94ED1E2224209216
:14151C00830306C000E20E94D91E81E0809383032224209202
:141530008102B19904C081E090E05C0102C0AA24BB242090C9
:14154400A5033324250142205320442019F4552009F452C0A4
:1415580005E00E9455021801442437FC4094552447FC509479
:14156C003092CD022092CC025092CF024092CE0280E991E427
:14158000AFE1B0E05A924A923A922A928C019D010E94E73CF7
:141594001093D1020093D0023093D3022093D202180130926E
:1415A8001B0320921A0320901A0330901B03232C3324288247
:1415BC002AE230E000270E947B030E94B40320901A033090D2
:1415D0001B0328822BE230E000270E947B030E94B403A89545
:1415E40000E80E94313C00E80E94313C8AE090E090932B03DA
:1415F80080932A0380912A0390912B038530E0E09E0708F4FC
:14160C0079CF0E94111C05E00E9455021801442437FC40944D
:14162000552447FC50943092CD022092CC025092CF02409280
:14163400CE0220901A0330901B03442455248090CE02909046
:14164800CF026090CC027090CD025A924A923A922A9283015C
:14165C0094010E94803D86E090E0A0E0B0E03A932A931A9369
:141670000A938C019D010E94803D1801290180E094E1A0E0A7
:14168400B0E0280E391E4A1E5B1E80E098E2A0E0B0E0BA931D
:14169800AA939A938A93810192010E94E73C1093D1020093D4
:1416AC00D0023093D3022093D20284E690E0A0E0B0E0BA9302
:1416C000AA939A938A930E94E73C0E948415A89500EA16E86A
:1416D40021E030E00E94493C0091D0021091D1020E948415B8
:1416E800A89500EA16E821E030E00E94493C002711270E9490
:1416FC0084150AC0A895B19903C00E94EE1504C00CEB10E0DD
:141710000E948415F5CFF8942CE230E000270E949403009329
:141724008303023018F40E94DB0103C000270E94DB017894FB
:141738000FE412E00E9406020DE00E9402022FE130E0002734
:14174C000E94940381E0801740F488832FE130E000270E9430
:141760007B030E94B4030E94011F8FEF9FEFAFEFB0E04090D2
:14177400CA025090CB022090C8023090C902281639064A0616
:141788005B0649F08FEF9FEFA3E0B0E082159305A405B50502
:14179C0088F58FEF88832BE130E000270E947B030E94B40377
:1417B00080E09CE0A0E0B0E09093C9028093C802B093CB025E
:1417C400A093CA022224288228E130E000270E947B030E9420
:1417D800B4038CE0888329E130E000270E947B030E94B40315
:1417EC0080E09CE088832AE130E000270E947B030E94B40347
:1418000081E080937C028FEF80937B02809321018093220169
:141814008093230180932401809325012BE130E000270E9433
:141828009403009383030F3FF9F422242092830328822BE18D
:14183C0030E000270E947B030E94B4032090830328822CE1FB
:1418500030E000270E947B030E94B4032090830328822DE1E6
:1418640030E000270E947B030E94B4030E94881F28E230E05D
:1418780000270E9494030093830324E630E08A010E94CD3C93
:14188C002090830333242016310681F024E630E08A010E9496
:1418A000CD3C00938303202E288228E230E000270E947B03B9
:1418B4000E94B40329E230E000270E9494030093830324E629
:1418C80030E08A010E94CD3C980104E610E00E94703D1A01E9
:1418DC00201A310A40908303552442145304B9F024E630E044
:1418F0008A010E94CD3C980104E610E00E94703D1A01201A97
:14190400310A20928303288229E230E000270E947B030E94AE
:14191800B40322242092830333C0809183038831C1F4222448
:14192C00209283030FC02224288220918303332700270E9456
:141940007B030E94B403809183038F5F809383038091830307
:14195400883168F31BC020918303332700270E949403202E51
:14196800332430921D0320921C03C1018F3FE0E09E0709F073
:14197C0009C0809183038F5F8093830380918303893148F2E5
:141990000E94111C05E00E94550220901803309019032016B9
:1419A400310678F409E412E00E9406020DE00E94020281E00F
:1419B8008093A7030E9407200E94200213C002E412E00E9484
:1419CC0006020DE00E94020281E0809378030E94C0208091EA
:1419E0006200877F809362000E94E1202DE230E000270E948B
:1419F40094030F3F09F0A7C18EE488832227332700270E94B0
:141A08007B030E94B40385E6888321E030E000270E947B0325
:141A1C000E94B40387E7888322E030E000270E947B030E94E9
:141A3000B40389E1888320E230E000270E947B030E94B403C4
:141A44002224288221E230E000270E947B030E94B40381E08A
:141A580088832FE130E000270E947B030E94B40381E0888343
:141A6C0026E230E000270E947B030E94B40381E0888327E239
:141A800030E000270E947B030E94B40381E088832DE230E017
:141A940000270E947B030E94B40381E088832EE230E00027EB
:141AA8000E947B030E94B40389E188832FE230E000270E9452
:141ABC007B030E94B40383E2888320E330E000270E947B0375
:141AD0000E94B4038AE1888321E330E000270E947B030E9436
:141AE400B40384E2888322E330E000270E947B030E94B40311
:141AF80081E0888323E330E000270E947B030E94B4038DE249
:141B0C00888324E330E000270E947B030E94B40387E388838E
:141B200025E330E000270E947B030E94B40381E0888327E383
:141B340030E000270E947B030E94B40381E0888328E330E066
:141B480000270E947B030E94B40381E0888329E330E000273A
:141B5C000E947B030E94B403222428822AE330E000270E9426
:141B70007B030E94B40381E088832BE330E000270E947B03B9
:141B84000E94B40381E088832CE330E000270E947B030E9480
:141B9800B40387EC88832DE330E000270E947B030E94B40344
:141BAC0087EC88832EE330E000270E947B030E94B4032224A0
:141BC00028822FE330E000270E947B030E94B40322242882B5
:141BD40020E430E000270E947B030E94B40382E0888321E4D7
:141BE80030E000270E947B030E94B40388E1888322E430E0AF
:141BFC0000270E947B030E94B40387EC888325E430E0002777
:141C10000E947B030E94B40387EC888326E430E000270E94E6
:141C24007B030E94B4032224288227E430E000270E947B0383
:141C38000E94B4032224288228E430E000270E947B030E944A
:141C4C00B40387EC888329E430E000270E947B030E94B40392
:141C600087EC88832AE430E000270E947B030E94B4032224EE
:141C740028822BE430E000270E947B030E94B40381E0888387
:141C88002CE430E000270E947B030E94B40385E088832DE407
:141C9C0030E000270E947B030E94B403222428822EE430E072
:141CB00000270E947B030E94B403222428822FE430E0002746
:141CC4000E947B030E94B4032224288220E530E000270E94C5
:141CD8007B030E94B4032224288221E530E000270E947B03D4
:141CEC000E94B40381E0888322E530E000270E947B030E941F
:141D0000B40381E0888323E530E000270E947B030E94B403F4
:141D140081E0888324E530E000270E947B030E94B40381E035
:141D2800888325E530E000270E947B030E94B40322242882F2
:141D3C0020E630E000270E947B030E94B4030E94FC1CF89497
:141D50000E94652178940AE312E00E9406020DE00E9402022F
:141D640004EF0E94020287E12090F204821578F08BE32090A7
:141D7800F104821550F08FE12090F304821528F08CE02090A9
:141D8C00F404821570F422242092F0042092F1042092F20415
:141DA00081E08093F5048093F4048093F304222484B78F712C
:141DB400281608F070C020E630E000270E9494030093830326
:141DC8002090F3042882202E86E0829D90012F593F4F002715
:141DDC000E947B030E94B4032090F40428822090830386E08C
:141DF000829D90012E593F4F00270E947B030E94B4032090CA
:141E0400F50428822090830386E0829D90012D593F4F0027A0
:141E18000E947B030E94B4032090F20428822090830386E051
:141E2C00829D90012C593F4F00270E947B030E94B40320908F
:141E4000F10428822090830386E0829D90012B593F4F00276A
:141E54000E947B030E94B40324B628822090830386E0829DC2
:141E680090012A593F4F00270E947B030E94B4031AE0009199
:141E7C0083030F5F0E94583D00938303202E288220E630E000
:141E900000270E947B030E94B40303E312E00E94060204B761
:141EA4000E94020280E884BF6CC28AE02090AC02821598F4C0
:141EB80022242092AC0280912001807F8093200120928703CF
:141ECC0020927E033324309229032092280320928203222430
:141EE00030906703231418F4A895209267032090AB02222089
:141EF40009F485C020905B0330905C03222019F4332009F4CC
:141F080070C08091F104853009F06BC02224332430925C03F8
:141F1C0020925B038091F604813009F060C020E230E0002793
:141F30000E9494032224201608F057C021E230E000270E94FD
:141F44009403013049F520E230E000270E94940300938303F8
:141F58002CE330E011270E94AD3C10931F0300931E031CE31B
:141F6C00009183030E945A3D00938303802F8F5F2090F104B6
:141F8000281A2092F10420901E0330901F038CE390E0821937
:141F940093098093F00427C020E230E000270E9494030093AA
:141FA80083032CE330E011270E94AD3C10931F0300931E0344
:141FBC001CE3009183030E945A3D009383033090F104300EB6
:141FD0003092F10420901E0330901F034090F0045524420C08
:141FE400531C4092F00481E08093B5020E943A05A895222425
:141FF8002092AB0281E0809335032090E303222029F1209028
:14200C00B5022220F1F12090AA022220A1F081E090E09093C2
:142020005C0380935B032090F30428822091F4040091A502AA
:142034001091A6020E940C0822242092AA0200270E947208B2
:142048000093830322242092B5021DC02090AA02222049F008
:14205C0081E090E090935C0380935B0322242092AA02209058
:14207000CF0380B3807182958F70821541F080B3807182954D
:142084008F708093CF030E94FC1C8091A9028130A9F42EE48E
:1420980030E000270E9494032224201668F42FE030E000913C
:1420AC002A0310912B030E94CB3C0030010711F40E94611823
:1420C0008091E203823069F480913503813009F05FC0009164
:1420D400AD03112717D522242092350357C02090CA033090A0
:1420E8007E02231440F480917D028F5F80937D0222242092F1
:1420FC007E0220906F0333244090220350902303421453042F
:1421100084F120906E03222061F12090370330907D02231431
:1421240018F4222420927D022090360330907D02231498F439
:142138002090CB0330907E02231410F445D524C02090C70322
:14214C00222011F445D51EC00091C7031127D6D419C020907A
:14216000CB0330907E02231410F432D511C036D50FC022242A
:1421740020927D022090CB0330907E02231410F425D504C06F
:142188000091C7031127BCD420905603222021F08091AC0304
:14219C00873C21F404EB0E94ED1E33C020903A03222021F484
:1421B0002090AC03222029F580915603813021F404EB0E949B
:1421C400D91E23C02090760330908002231450F4222420924F
:1421D800800204EB0E94D91E81E08093630313C02090770312
:1421EC0030908002231468F404EB0E94ED1E22242092630310
:1422000006C004EB0E94ED1E22242092630320903B032220DA
:1422140009F47AC020903903222029F42090AB03222009F09B
:142228006EC080915503813021F405EB0E94D91E69C02090E3
:14223C00560330905503321421F480913A03813029F02090FA
:14225000AC03222009F03AC080915503833079F480915403A5
:14226400815020906303282621F005EB0E94D91E4BC005EB9C
:142278000E94ED1E47C082E080935503882309F441C0209078
:14228C008002222021F480915403813041F0809180028B30CD
:1422A00059F480915403823039F4222420927F0205EB0E948B
:1422B400D91E2AC02090750330907F02231420F505EB0E94EE
:1422C800ED1E20C080915503823011F08330D1F4209074035C
:1422DC0030907F02231438F4222420927F0205EB0E94D91E48
:1422F0000DC02090750330907F02231438F405EB0E94ED1EA4
:1423040003C005EB0E94ED1E809134038130F1F42090800354
:14231800222011F037D018C084E020908102821598F422248F
:14232C00209280032092C9032092C70384E18093CB038AE0BE
:142340008093CA0300271127DFD32224209281020E94562005
:14235400222420927C0320907A03222039F0222420927A03F1
:142368000E94313B0E94833B20908603222031F0A8950E9478
:14237C00FC352224209286030BD693CD219608950E94C23D65
:14239000222420928102209280032DE230E000270E9494030A
:1423A400073C09F05CC081E080936403A8952090850322203B
:1423B800E9F422242092C90380EA809385030E94FB3E9801F7
:1423CC002F71307004E610E00E94703DC80188539F4F9093DF
:1423E00027038093260324E630E08C010E94CD3C00937F031C
:1423F40080918503815080938503843600F515E0082F0E9453
:142408005A3D20907F03209E80012AE030E00E94B13C20905F
:14241C00260330902703201A310A309227032092260324E653
:1424300030E081010E94CD3CC80147968093C90310C08091F5
:1424440085038C3860F424E630E000912603109127030E94A3
:14245800CD3CC80147968093C90322243090C903231438F4AD
:14246C00232C2092620388E0809361030DC0222430906103E0
:14248000231428F4832D81508093610303C0222420926203DD
:1424940020907103222041F020906203332430922103209299
:1424A800200307C02090C90333243092210320922003809197
:1424BC006D038F5F80936D0318E0082F0E94583D00936D03C2
:1424D000209020033090210387ED93E0E02FFF27E80FF91F16
:1424E400208220926B032092570382E080936A0381E08093C0
:1424F800690320906D032092680380938303B2C02090680301
:14250C00222019F488E08093680380916803815080936803BB
:1425200087ED93E0E0916803FF27E80FF91F208020926003FA
:14253400E0916803FF27E80FF91F20803324321408F088C005
:1425480020905703222041F4E0916803FF27E80FF91F20804D
:14255C002092570387ED93E0E0916803FF27E80FF91F2080C7
:1425700030906B03231431F4809169038F5F8093690360C0C3
:1425840087ED93E0E0916803FF27E80FF91F208030906B037D
:14259800321420F481E08093650303C022242092650387ED62
:1425AC0093E0E0916803FF27E80FF91F208020925D03209035
:1425C0006B03332400915D031127021913090E94993C81E00A
:1425D40090E08017910784F48093690382E080936A0387ED07
:1425E80093E0E0916803FF27E80FF91F20802092570324C0CB
:1425FC0080916A03823051F42090650320926A0380916903A2
:142610008F5F8093690316C02090650380916A03820D81309D
:1426240051F482E08093690320926A0320906B032092570333
:1426380005C0809169038F5F8093690387ED93E0E09168031C
:14264C00FF27E80FF91F208020926B0380916903853009F456
:142660000AC0809183038F5F8093830380918303883008F433
:1426740049CF80916903853050F02090570320925F032092F8
:14268800720386E080935E0324C0222420925F0320902203DC
:14269C00309023030091200310912103021913090E94993C1D
:1426B0000230E0E01E0724F486E080935E030DC081E020902F
:1426C4005E03821528F4822D815080935E0303C0222420923F
:1426D800720380913803823000F5222430907203231490F450
:1426EC0020905803321451F088E080933803232C332430922A
:1427000023032092220312C081E0809338030EC02224209281
:1427140038033324309223032092220305C08091380381507E
:14272800809338032090240330902503409022035090230395
:14273C004218530881E090E08415950514F45C0102C0AA24DB
:14275000BB24209124033091250385010E94703D00300107C8
:14276400F1F420902203309023034090240350902503421868
:14277800530882E090E0841595051CF481E05C0102C0AA248F
:14278C00BB24209124033091250385010E94703D003001078C
:1427A00021F0009124030E94D33920903803222019F0822DC9
:1427B400883011F5209059032220C1F020907003332440900A
:1427C8002203509023034214530439F4209024033090250339
:1427DC002092C7030DC020902203309023032092C70306C0A3
:1427F00020902203309023032092C703222430905903231405
:1428040028F4832D8150809359031CC02224209270032090BD
:142818002203309023030091240310912503021913090E9447
:14282C00993C0130E0E01E0749F48FE08093590320902403BB
:142840003090250320927003209022033090230330922503D2
:14285400209224032090CE033324409022035090230342146E
:142868005304B4F181E08093B0032090CD03332442145304B5
:14287C0004F12090CC033324421453046CF082E08093CB0331
:1428900085E08093CA0384E08093360389E08093370320C0A9
:1428A40083E08093CB0387E08093CA0384E08093360388E07D
:1428B8008093370313C086E08093CB038AE08093CA0383E0F8
:1428CC008093360386E08093370306C084E18093CB038AE083
:1428E0008093CA032090AC03332440902203509023034214FD
:1428F4005304C4F081E080933A03809156038330A1F42090B2
:14290800B0033090CB03329C009277033090CA03329C0092B3
:14291C00760320907E022092800203C0222420923A03209022
:14293000AB033324409022035090230342145304C4F081E0D1
:1429440080933903809155038330A1F42090B0033090CB038E
:14295800329C009275033090CA03329C0092740320907E02FF
:14296C0020927F0203C02224209239032090D603332440907D
:142980002203509023034214530494F08091D503813031F428
:1429940022242092C7032092C80308C08091D503823021F478
:1429A8002090AD032092C703209064033324409022035090FC
:1429BC002303421453041CF422242092C7038091E2038330B9
:1429D00021F42090AD032092C7030E94B03D08950E94C93D2E
:1429E400C22EE02EAE8084EB93E0EE2DFF27E80FF91F2080E1
:1429F8002092B203EC2DFF27E80FF91F20802092B1038091FF
:142A0C006200806880936200DF9A2090B20325BA2090B103D6
:142A20002BBA22242092810201C0A895209081022A14D8F308
:142A34002224209281020027112764D00E94BF3D08950E94A3
:142A4800C53DA22EC02EA89514E60C2D0E945A3D00938303F8
:142A5C0084EB93E0E02FFF27E80FF91F20802092B303202EEA
:142A70008AE0829D10012AE030E00C2D11270E94B13C280175
:142A84004218530850921F0340921E0384EB93E0F201E80FC6
:142A9800F91F20802092B2032090830384E6829DEC2DFF270D
:142AAC00E019F10992010AE010E00E94703DE01BF10B84EB01
:142AC00093E0E80FF91F20802092B10380916200806880930C
:142AD4006200DF9A2090B20325BA2090B1032BBA222420928E
:142AE800810201C0A895209081022A14D8F3222420928102A2
:142AFC000027112703D00E94BC3D08950E94C23D5801A09230
:142B10005803AA2049F4BB2039F45AD0809162008F77809391
:142B2400620043C024E630E085010E94B13C0093830384EB81
:142B380093E0E02FFF27E80FF91F20802092B303202E8AE012
:142B4C00829D10012AE030E085010E94B13C28014218530838
:142B600050921F0340921E0384EB93E0F201E80FF91F2080E6
:142B74002092B2032090830384E6829DF501E019F1099201AB
:142B88000AE010E00E94703DE01BF10B84EB93E0E80FF91F28
:142B9C0020802092B1038091620080688093620003D00E94DA
:142BB000B03D0895DF9A2090AE03222039F02090B20325BAFE
:142BC4002090B1032BBA01C001D00895DF9A8FE785BB8FEFD8
:142BD8008BBB08952090AE03222049F08091620080688093BC
:142BEC00620022242BBA25BA01C0ECDF08950E94C23D2197E7
:142C0000A89581E08093AE03AA2439C084EB93E0EA2DFF2778
:142C1400E80FF91F20802092B2032092B3032AE030E00A2DDD
:142C280011270F5F1F4F0E94AD3CF80184EB93E0E80FF91F0F
:142C3C0020802092B1032AE030E00A2D11270F5F1F4F0E9477
:142C5000AD3C18018AE08A9D8001020D131D54DF08EA11E601
:142C640020E030E00E94493CB1DF00E117E220E030E00E9409
:142C7800493CA895A3948A2D8A3008F4C3CF2BE430E000270A
:142C8C000E9494030023B1F000E21EE420E030E00E94493C1C
:142CA000A8959CDF00E711E121E030E00E94493C8FDF00E108
:142CB40017E220E030E00E94493CA8951A9878940E949802A5
:142CC800222420927E023324309229032092280380916200EB
:142CDC0081608093620001C0A89580917E028834D8F3222432
:142CF00020927E0281B18071809383032090830381B1807189
:142D0400821521F480917E028230B0F380917E02823098F559
:142D18000E94A702222420927E0219C02090830381B18071B2
:142D2C00821599F080912803909129030196909329038093F1
:142D400028032090830381B18071821521F020907E022220E1
:142D5400B1F320907E02222019F3009128031091290301506F
:142D68001040CEDEA89500EF19E422E030E00E94493CA895BC
:142D7C0005C088E2888321E00EE02CDE809162008E7F80937D
:142D900062000E946A021A9A00271127B5DE21960E94B03DD3
:142DA400089580EC8093B40389EF8093B50384EA8093B603CB
:142DB80080EB8093B70389E98093B80382E98093B90382E8EB
:142DCC008093BA0388EF8093BB0380E88093BC0380E9809325
:142DE000BD0388E88093BE0383E88093BF0386EC8093C00353
:142DF40081EA8093C10386E88093C2038EE88093C3038CE880
:142E08008093C4038FEF8093C5038093C60308950E94C53D66
:142E1C00C22EA02E26978AE090E0998388832C2D33278E01E4
:142E30000E5F1F4F0E949B3E0A810E9402022B80222019F011
:142E4400022D0E9402020FE20E9402028AE090E0998388830D
:142E58002A2D33278E010E5F1F4F0E949B3E0A810E9402029F
:142E6C002B80222019F0022D0E9402020FE20E9402028AE086
:142E800090E0998388832A8533272053384F8E010E5F1F4F3A
:142E94000E949B3E0A810E9402020B810E9402020C810E941D
:142EA80002020D810E94020226960E94BC3D08950E94C53D46
:142EBC00A22EC02E26978AE090E0998388832C2D33278E0144
:142ED0000E5F1F4F0E949B3E2A80222019F400E30E94020216
:142EE4002A80222019F0022D0E9402022B80222019F0022DEB
:142EF8000E9402020AE30E9402028AE090E0998388832A2D35
:142F0C0033278E010E5F1F4F0E949B3E2B80222019F400E395
:142F20000E9402022A80222019F400E30E9402022A80222089
:142F340019F0022D0E9402022B80222019F0022D0E940202E0
:142F48000AE30E9402028AE090E0998388832A8533278E0149
:142F5C000E5F1F4F0E949B3E2B80222019F400E30E94020288
:142F70002A80222019F400E30E9402022A80222019F0022DA7
:142F84000E9402022B80222019F0022D0E94020226960E946A
:142F9800BC3D08950C9936C081E080937C030BEF10E031D016
:142FAC0022242092A60320927B020C9929C02092810315C0A8
:142FC00007EF11E024D01091810301B1007102950F700E9422
:142FD4002C3E2090A603202A2092A603809181038F5F8093EB
:142FE800810380918103883038F307EF11E00BD00C9B08C0A8
:142FFC002090A60320927B02022D0AD000E2D3D6089502C046
:143010000150104000300107D9F708950F3321F00B3211F0D5
:143024000D3231F481E08093D30322242092D2032090D30397
:143038002220B1F12090D203222019F40093D1030EC0809186
:14304C00D203843050F485EE93E0E091D203FF27E80FF91F42
:14306000802F805380838091D2038F5F8093D2038530D1F4A1
:1430740022242092E9032092D2032092D30381E0809380035E
:143088002090E7038AE0829D10014090E60384E6849D402C50
:14309C00420C2090E803420C4092C90308950E94F23D0E943B
:1430B000ED070093EA030E94BE03A8950E94093E18952797A4
:1430C40000E475D605EB73D6222420920201209294020E94AB
:1430D800D40722242092810201C0A895809181028F3F20F41A
:1430EC00209002012220B9F380919402813471F020902C0393
:1431000030902D0340902A0350902B034214530418F40E9465
:14311400E50783C308E112E00E94060220900201222009F4FE
:14312800F9C22090E503222009F47FC0009194020E940202F5
:14313C000AE00E9402020CEF11E00E9406020AE00E940202C9
:143150000AE00E9402020FED11E00E9406020AE00E940202B4
:143164000FEC11E00E94060220909002288220918F02009102
:143178008E024EDE0AE00E94020207EC11E00E9406022090B9
:14318C009302288220919202009191028FDE809194028635B8
:1431A00031F488E2888324E00EE01ADC1DC38091940281345D
:1431B40031F088E2888325E00EE010DC13C324E100918F0295
:1431C8003EDC01C0A895809181028230D8F324E100918E02A4
:1431DC0034DC01C0A895809181028230D8F324E10091900298
:1431F0002ADC01C0A895809181028630D8F324E10091910289
:1432040020DC01C0A895809181028230D8F324E10091920281
:1432180016DC01C0A895809181028230D8F324E10091930276
:14322C000CDCA895DBC280919402813409F0ADC120909202C5
:143240002092F104209093022092F00420908E022092F304FF
:1432540020908F022092F404209090022092F504822D99271F
:143268008053984F9093A6028093A5022DE430E000270E9429
:14327C009403802F8078803809F03FC00E948106202E2DE4C8
:1432900030E000272F920E9494032F9040909102420C802FDA
:1432A4008F77480E242C2092830387E1841508F52090F3048D
:1432B80028822091F4040091A5021091A6020E94ED06980100
:1432CC002F5F3F4F8E010F5F1F4F0E943F078D819E81805D75
:1432E00097408093F5042B803C802092F40429803A802092D1
:1432F400F30418E1009183030E94583D0093F2045CC02DE4D2
:1433080030E000270E949403802F8F7790919102985E981B2F
:14331C00292E20928303983108F040C02090F304288220914B
:14333000F4040091A5021091A6020E94ED0698012150304001
:143344008E010F5F1F4F0E943F0718E1009183030E94583DDB
:143358000093F2040E9481062090F204200E87E1821580F468
:14336C0029803A8028822B810D811E810E94ED0698012F5FAB
:143380003F4F8E010F5F1F4F0E943F078D819E81805D974077
:143394008093F5042B803C802092F40429803A802092F304FC
:1433A8000E948106202E00918303020D18E10E94583D0093B1
:1433BC00F2042090E303222079F02090F30428822091F404CC
:1433D0000091F50411270053184F0E940C0801E00E947208BA
:1433E40001E40E9402020AE00E9402020CEF11E00E94060224
:1433F8000AE00E9402020AE00E9402020FED11E00E9406020A
:14340C000AE00E9402020FEC11E00E9406022090900228829A
:1434200020918F0200918E02F7DC0AE00E94020207EC11E0EE
:143434000E940602209093022882209192020091910238DD6D
:143448000AE00E9402020AE00E9402020CEA11E00E940602BF
:14345C000AE00E9402020FEC11E00E9406022090F5042882E3
:143470002091F4040091F304CFDC0AE00E94020207EC11E0F8
:143484000E9406022090F00428822091F1040091F20410DD22
:143498000AE00E9402022090F50428822090F60485E0829D0F
:1434AC0090012550304020563F4F00270E947B030E94B403F2
:1434C0002090F40428822090F60485E0829D90012550304002
:1434D4002F553F4F00270E947B030E94B4032090F3042882E1
:1434E8002090F60485E0829D9001255030402E553F4F0027F4
:1434FC000E947B030E94B4032090940228822090F60485E044
:14351000829D9001255030402D553F4F00270E947B030E9419
:14352400B40381E088832090F60485E0829D900125503040CC
:143538002C553F4F00270E947B030E94B4032090A703222034
:14354C0009F44CC13FDB00E513EC20E030E00E94493C84E1C7
:14356000888326E002E13CDA84E1888320E102E137DA84E183
:14357400888325E002E132DA88E2888321E002E12DDA24DBE5
:1435880000E513EC20E030E00E94493C29C1809194028635C8
:14359C0009F060C005E40E94020204E30E9402022090F5043D
:1435B00028822090F60485E0829D90012550304020563F4FB5
:1435C40000270E947B030E94B4032090F40428822090F60457
:1435D80085E0829D9001255030402F553F4F00270E947B038C
:1435EC000E94B4032090F30428822090F60485E0829D900162
:14360000255030402E553F4F00270E947B030E94B403209070
:14361400940228822090F60485E0829D9001255030402D553C
:143628003F4F00270E947B030E94B40384E088832090F60447
:14363C0085E0829D9001255030402C553F4F00270E947B032A
:143650000E94B40388E2888324E00EE0C1D9C4C005E40E94FD
:14366400020205E30E9402022090F50428822090F60485E05E
:14367800829D90012550304020563F4F00270E947B030E94BC
:14368C00B4032090F40428822090F60485E0829D90012550ED
:1436A00030402F553F4F00270E947B030E94B4032090F3044D
:1436B40028822090F60485E0829D9001255030402E553F4FA3
:1436C80000270E947B030E94B40385EE88832090F60485E0C1
:1436DC00829D9001255030402D553F4F00270E947B030E944C
:1436F000B40385E088832090F604829D9001255030402C55DF
:143704003F4F00270E947B030E94B40388E2888325E00EE01B
:1437180063D966C009EA11E00E9406020AE00E94020206E82F
:14372C0011E00E9406020AE00E9402022090F504288220905B
:14374000F60485E0829D90012550304020563F4F00270E94B4
:143754007B030E94B4032090F40428822090F60485E0829D0A
:143768009001255030402F553F4F00270E947B030E94B40325
:14377C002090F30428822090F60485E0829D90012550304044
:143790002E553F4F00270E947B030E94B40383EE8883209048
:1437A400F60485E0829D9001255030402D553F4F00270E9444
:1437B8007B030E94B40383E088832090F60485E0829D9001F9
:1437CC00255030402C553F4F00270E947B030E94B40388E2EB
:1437E000888323E00EE0FCD822242092320320923103209240
:1437F400330320922E0320922F032092300300E4EAD205EB4F
:14380800E8D20E94E50722242092E5032092A90204EF0E9492
:14381C000202279608952AE230E000270E949403202E332419
:14383000442455243092D1022092D0025092D3024092D2022D
:1438440088E090E08A93810192010E94203E10931F0300930E
:143858001E032BE230E000270E94940300938303202E332400
:14386C0040901E0350901F03420C531C50921F0340921E03A1
:14388000C2018839E8E09E0728F084E59BE08415950538F4E8
:1438940080E09AE090931B0380931A0308C020901E0330907C
:1438A8001F0330921B0320921A0320901A0330901B03442428
:1438BC0055243092C1022092C0025092C3024092C202409079
:1438D000C2025090C3022090C0023090C10284E690E0A0E02C
:1438E400B0E05A924A923A922A928C019D010E94803D86E000
:1438F80090E0A0E0B0E03A932A931A930A938C019D010E949B
:14390C00803D1801290180E092E0A0E0B0E0280E391E4A1ED0
:143920005B1E8AE090E08A93810192010E94323E1093C10296
:143934000093C0023093C3022093C20280EE98ECA0E1B0E028
:143948003A932A931A930A938C019D010E94E73C1093D10231
:14395C000093D0023093D3022093D20218013092190320922A
:1439700018034090C2025090C3022090C0023090C10280E199
:143984009DECAEE0B0E05A924A923A922A928C019D010E946B
:14399800E73C1093D1020093D0023093D3022093D2021801E5
:1439AC0030921703209216034090C2025090C3022090C002B5
:1439C0003090C10288EA97E0AFE0B0E05A924A923A922A9218
:1439D4008C019D010E94E73C1093D1020093D0023093D3027C
:1439E8002093D2021801309215032092140308950E94C23D4A
:1439FC002197A89521E530E000270E949403002359F020E5DB
:143A100030E000270E949403002321F081E090E05C0102C00E
:143A2400AA24BB24A092E30328E430E000270E949403202EFF
:143A38002BE430E000272F920E9494032F90209E00926E03BA
:143A4C0023E330E000270E9494030093D50327E330E0002744
:143A60000E9494030093E2032CE330E000270E94940300938F
:143A7400A7032FE330E000270E9494030093560320E430E012
:143A880000270E9494030093550321E430E000270E9494036A
:143A9C000093540327E430E000270E949403009371032FE497
:143AB00030E000270E9494030093E10381E080933503A0903F
:143AC4005603BB24AA2011F4BB2051F0C5018130E0E09E07EF
:143AD80061F08230E0E09E0779F01BC022242092770389E152
:143AEC008093760317C084E1809377038AE08093760310C0AB
:143B00002CE430E000270E949403802F865F8093770385E1AA
:143B14008093760303C0222420927703A0905503BB24AA20AB
:143B280011F4BB2051F0C5018130E0E09E0761F08230E0E0C9
:143B3C009E0779F01BC022242092750389E18093760317C04F
:143B500084E1809375038AE08093740310C02CE430E0002766
:143B64000E949403802F865F8093750385E18093740303C042
:143B78002224209275032090E303222009F0FAC02AE330E021
:143B8C0000270E949403002309F45FC02090CF03222009F0C9
:143BA0005AC020E330E000270E9494030093AD0322E330E02C
:143BB40000270E9494030093CE03202E87E6829D8001005787
:143BC8001E4F24E630E00E94B13C0093CD032090CE038EE67B
:143BDC00829D800106571D4F24E630E00E94B13C0093CC0361
:143BF00025E330E000270E9494030093D60326E430E000279C
:143C04000E9494030093AC032EE330E000270E94940300931D
:143C1800AB032EE230E000270E949403009364032AE430E052
:143C2C0000270E94940300936F0323E530E000270E949403A7
:143C40000093AE0325E530E000270E9494030093AF03A89530
:143C540059C02FE230E000270E9494030093AD0321E330E06B
:143C680000270E9494030093CE03202E87E6829D80010057D2
:143C7C001E4F24E630E00E94B13C0093CD032090CE038EE6C6
:143C9000829D800106571D4F24E630E00E94B13C0093CC03AC
:143CA40024E330E000270E9494030093D60325E430E00027E9
:143CB8000E9494030093AC032DE330E000270E94940300936A
:143CCC00AB032DE230E000270E9494030093640329E430E0A0
:143CE00000270E94940300936F0322E530E000270E949403F4
:143CF4000093AE0324E530E000270E9494030093AF03A8957D
:143D0800222430905503231478F42EE430E000270E94940324
:143D1C00002341F48091AB03873C20F481E090E05C0102C0B5
:143D3000AA24BB24A0923B0320905503222021F08091AB0348
:143D4400873C11F405EB47D08091E203813011F0833069F4E4
:143D58002090AE03222021F42090AF03222029F01A9A81E0CD
:143D6C008093340313C01A982224209234030EC02090F304D0
:143D800028822091F4040091A5021091A6020E940C0801E0C4
:143D94000E9472082090AE03222029F4809162008F778093B3
:143DA800620021960E94B03D0895043B11F4C59A0FC0053B10
:143DBC0011F4C49A0BC0003211F4959807C0003411F4969833
:143DD00003C0003809F497980895043B11F4C5980FC0053B6B
:143DE40011F4C4980BC0003211F4959A07C0003411F4969A09
:143DF80003C0003809F4979A089528E130E000270E94940378
:143E0C00202E3324442455243092D1022092D0025092D3024C
:143E20004092D20288E090E08A93810192010E94203E10933B
:143E3400C9020093C8023093CB022093CA0288E090E08A934E
:143E48000E94203E1093C9020093C8023093CB022093CA028C
:143E5C0029E130E000270E949403202E332444245524309290
:143E7000D1022092D0025092D3024092D20288E090E08A9395
:143E8400810192010E94203E1093D1020093D0023093D302A2
:143E98002093D2028090CA029090CB026090C8027090C90241
:143EAC00600E711E821E931E7092C9026092C8029092CB023C
:143EC0008092CA022AE130E000270E949403202E3324442488
:143ED40055243092D1022092D0025092D3024092D2028090DB
:143EE800CA029090CB026090C8027090C902620C731C841CEB
:143EFC00951C7092C9026092C8029092CB028092CA0208950E
:143F10002BE130E000270E949403202E3324442455243092D9
:143F2400D1022092D0025092D3024092D20288E090E08A93E0
:143F3800810192010E94203E1093C5020093C4023093C70211
:143F4C002093C60288E090E08A930E94203E1093C5020093F4
:143F6000C4023093C7022093C6022CE130E000270E94940303
:143F7400202E3324442455243092D1022092D0025092D302E3
:143F88004092D20288E090E08A93810192010E94203E4090A5
:143F9C00C6025090C7022090C4023090C502200E311E421EC6
:143FB000531E3092C5022092C4025092C7024092C6022DE138
:143FC40030E000270E949403202E3324442455243092D1025E
:143FD8002092D0025092D3024092D2028090C6029090C70233
:143FEC006090C4027090C502620C731C841C951C7092C5022D
:144000006092C4029092C7028092C6020895219785B78F7D92
:1440140085BFA89589E88093610088E08093620000EA16E86D
:1440280021E030E00E94493CA8952AD10E94E81500E8BBDEF4
:14403C0000EA16E821E030E00E94493CA895222420927803A0
:1440500005E00E943B02D5DE5BDF1A9A00EA16E821E030E0FE
:144064000E94493CA8952090A703222011F00E94FD15C0DCF7
:144078002224332430922B0320922A032090E303222071F08F
:14408C002090F30428822091F4040091A5021091A6020E9403
:1440A0000C0801E00E9472082196089580917B03813039F43A
:1440B4000E94480200E28FDE222420927B03349B5CC00E94BA
:1440C8004B0220901603309017030215130508F052C0222475
:1440DC002092C703809162008F7780936200332430922B031F
:1440F00020922A0320928303A89580912A0390912B0381302A
:14410400E0E09E07C0F305E00E945502209014033090150312
:144118000215130580F530D0A8950FC0209083033324409086
:14412C002A0350902B032414350428F4822D8F5F8093830381
:14414000A89580912A0390912B038A30E0E09E0748F3A8950A
:1441540005E00E94550220901403309015030215130550F467
:1441680081E08093780380916200877F8093620024D001C0B1
:14417C0048DF08951A980E94313B0E94833B22242ABA27BA40
:1441900024BA21BA22B888E080936100209264002BBA8FE43E
:1441A40088BB25BA22BA23B884E5809362008EE18093650069
:1441B8000E94E5070E944602089585B7886185BF85B7806257
:1441CC0085BF0E944602A89557C08895A8952090AB02222064
:1441E00029F00E943A0522242092AB021AE00091F0040E940B
:1441F400583D002309F03FC005E00E9455022090180330909E
:1442080019032016310698F589E88093610088E080936200CA
:14421C002224332430922B0320922A03209283030FC020906B
:144230008303332440902A0350902B032414350428F4822D56
:144244008F5F80938303A89580912A0390912B038A30E0E09B
:144258009E0748F305E00E94550220901803309019032016B7
:14426C00310610F4CEDE01C085DF0E944602209078032220DB
:1442800009F401C0A8CF08958FEF8ABB81EB87BB8FEF84BB2A
:144294008BEE81BB8EE482B92224209264002BBA8CE488BBC0
:1442A80025BA84E182BB0E94E507222423B88CE580936200EC
:1442BC0087E080936500959A969A979A0895A89581B5886186
:1442D00081BDA8958FE081BD0895A89581B5886181BD222435
:1442E40021BCA89508950E94F23D0E94FE0122242092AC02F7
:1442F80003D00E94093E18950E94C23D2897A8952090870372
:14430C00222011F40C94E029A22CBB24C5018E3CE0E09E070B
:1443200009F4DAC48EEC8A159B050CF432C0C501803BE0E002
:144334009E0709F44CC0813BE0E09E0709F447C0823BE0E025
:144348009E0709F442C0833BE0E09E0709F40CC1843BE0E051
:14435C009E0709F407C1853BE0E09E0709F402C1803BE0E083
:144370009E0714F40C949935C501883CE0E09E0709F4EEC183
:144384008B3CE0E09E0709F470C30C949935C5018D3EE0E00A
:144398009E0709F408C68DEE90E08A159B0544F0C501863EB9
:1443AC00E0E09E0709F4EFC60C949935C5018D3FE0E09E0781
:1443C00009F471C58E3FE0E09E0709F46BC60C949935209038
:1443D400200133242094309422FE2CC08EEE93E0E09128034E
:1443E800F0912903E80FF91F20907B02208220907B02309049
:1443FC007F03322430927F0380912803909129038F3FE0E07A
:144410009E0739F4809120018460809320010C9499358091FD
:14442400280390912903019690932903809328030C9499357A
:144438002090200133242094309423FE1CC080917B02813F85
:14444C0071F48091200188608093200120907B0230907F033A
:14446000322430927F030C94993580912001807F80932001DB
:1444740003EF0E9402020C94993520907B0230907F03321479
:1444880009F048C08EEE93E0998388832091ED0300270E949F
:14449C0056030E94B4038091ED038F5F8093ED038091EC0368
:1444B00081508093EC032224332430922903209228038091AC
:1444C4002001807F8093200120927F032090EC032220E9F49E
:1444D8002090E303222079F02090F30428822091F404009104
:1444EC00F50411270053184F0E940C0801E00E9472082224D8
:1445000020928703332430922903209228032092820302EF21
:144514000E9402020C94993503EF0E9402028091EB03815017
:144528008093EB03882389F480912001807F809320012224AB
:14453C002092870333243092290320922803209282030C9436
:14455000993580912001807F80932001222433243092290399
:144564002092280320927F030C94993580917B02813F49F439
:1445780030907F03382630927F0381E0809388031FC080915C
:14458C0088038130D9F420907B0230907F03321469F02224BE
:1445A00020927E0320927F03209288032092870303EF0E9493
:1445B400020208C081E080937E03222420927F03209288037B
:1445C80080917E03813009F03FC02090200133242094309404
:1445DC0022FE38C0A89580918703833B61F480E091E09093D4
:1445F0001D0380931C03809120018460809320011FC080912B
:144604008703843B61F480E094E090931D0380931C038091AA
:1446180020018460809320010FC080918703853B59F480E07E
:14462C0099E090931D0380931C038091200184608093200142
:1446400002EF0E9402020E94B40300EF0E94020280917E034F
:14465400813011F00C9499352090200122FE01C002C00C941E
:14466800993580917B02823F81F48091EC0381508093EC03D9
:14467C0080911C0390911D0380509F4F90931D0380931C0386
:1446900009C080917B02833F29F48091EB0381508093EB030F
:1446A40022243090EC03231408F04AC03090EB03231408F0F7
:1446B80045C020901C0330901D0330921F0320921E031AC0A9
:1446CC0020911E0330911F0300270E949403009383033090EC
:1446E0007F03302630927F030E940202A89580911E03909174
:1446F4001F03019690931F0380931E0380911C0390911D030F
:1447080080509F4F20901E0330901F0328163906C8F281EF85
:14471C0090E020907F0333242826392620927F0301EF0E941D
:14473000020200917F030E940202222420927F030C949935D0
:1447440080912001807F80932001222420927E0320927F034F
:14475800209287030C94993580912803909129030196909360
:14476C00290380932803A8958130E0E09E070CF46FC18AE1E1
:1447800090E02090280330902903821593050CF465C1910107
:1447940002E010E00E94703DF8018AE890E0E80FF91F059071
:1447A8001490F001099420907B0220923C0352C120907B026D
:1447BC0020923D034DC120907B0220923E0348C120907B0293
:1447D00020923F0343C120907B02209240033EC120907B028F
:1447E4002092410339C120907B022092420334C120907B028B
:1447F800209243032FC120907B02209244032AC120907B0287
:14480C002092450325C120907B022092460320C120907B0282
:14482000209247031BC120907B022092480316C120907B027E
:144834002092490311C120907B0220924A030CC120907B027A
:1448480020924B0307C120907B0220924C0302C120907B0276
:14485C0020924D03FDC020907B0220924E03F8C020907B0274
:1448700020924F03F3C020907B0220925003EEC020907B0270
:1448840020925103E9C020907B0220925203E4C020907B026C
:1448980020925303DFC020907B0230907F03321409F0CDC02A
:1448AC0020903C0328822FE230E000270E947B030E94B4039E
:1448C00020903D03288220E330E000270E947B030E94B40397
:1448D40020903E03288221E330E000270E947B030E94B40381
:1448E80020903F03288222E330E000270E947B030E94B4036B
:1448FC0020904003288224E330E000270E947B030E94B40354
:1449100020904103288225E330E000270E947B030E94B4033D
:144924002090420328822DE230E000270E947B030E94B40321
:144938002090430328822EE230E000270E947B030E94B4030B
:14494C0020904403288225E430E000270E947B030E94B403FD
:1449600020904503288226E430E000270E947B030E94B403E7
:144974002090460328822DE330E000270E947B030E94B403CC
:144988002090470328822EE330E000270E947B030E94B403B6
:14499C00A89520904803288221E430E000270E947B030E9427
:1449B000B40320904903288229E430E000270E947B030E9490
:1449C400B40320904A0328822AE430E000270E947B030E947A
:1449D800B40320904B03288222E530E000270E947B030E946C
:1449EC00B40320904C03288223E530E000270E947B030E9456
:144A0000B40320904D03288224E530E000270E947B030E943F
:144A1400B40320904E03288225E530E000270E947B030E9429
:144A2800B4030E94FC1C2224332430922903209228032092EF
:144A3C00870302EF0E9402020BC003EF0E9402022224332445
:144A500030922903209228032092870320907B0230907F03DC
:144A6400322430927F030C9499358091280390912903019616
:144A780090932903809328038130E0E09E070CF41EC182E145
:144A8C0090E02090280330902903821593050CF414C1910149
:144AA00002E010E00E94703DF8018EEB90E0E80FF91F05905B
:144AB4001490F001099420907B0220923C0301C120907B02AF
:144AC80020923D03FCC020907B0220923E03F7C020907B0228
:144ADC0020923F03F2C020907B0220924003EDC020907B0224
:144AF00020924103E8C020907B0220924203E3C020907B0220
:144B040020924303DEC020907B0220924403D9C020907B021B
:144B180020924503D4C020907B0220924603CFC020907B0217
:144B2C0020924703CAC020907B0220924803C5C020907B0213
:144B400020924903C0C020907B0220924A03BBC020907B020F
:144B540020924B03B6C020907B0230907F03321409F0A4C0C5
:144B680020903E032092D503288223E330E000270E947B03B7
:144B7C000E94B403209040032092830328822AE330E00027B3
:144B90000E947B030E94B403209041032092560328822FE3DD
:144BA40030E000270E947B030E94B40320904203209255034E
:144BB800288220E430E000270E947B030E94B4032090430395
:144BCC0020927103288227E430E000270E947B030E94B4034A
:144BE000209044032092A70328822CE330E000270E947B035E
:144BF4000E94B4032090450320928303288228E430E0002737
:144C08000E947B030E94B403209047032092830328822DE432
:144C1C0030E000270E947B030E94B4032090480320928303A1
:144C3000288221E530E000270E947B030E94B4032090490314
:144C440020928303288221E430E000270E947B030E94B403C5
:144C580020904A032092830328822CE430E000270E947B0302
:144C6C000E94B4030E94FC1C2090E303222071F02090F30441
:144C800028822091F4040091A5021091A6020E940C0801E0B5
:144C94000E947208222433243092290320922803209287034C
:144CA80002EF0E9402020BC003EF0E9402022224332430929F
:144CBC002903209228032092870320907B0230907F033224DA
:144CD00030927F030C949935809128039091290301969093DB
:144CE4002903809328038130E0E09E070CF4D0C082E190E0D9
:144CF8002090280330902903821593050CF4C6C0910102E0B8
:144D0C0010E00E94703DF80182EE90E0E80FF91F0590149033
:144D2000F001099420907B0220923C03B3C020907B02209281
:144D34003D03AEC020907B0220923E03A9C020907B02209255
:144D48003F03A4C020907B02209240039FC020907B02209251
:144D5C0041039AC020907B022092420395C020907B0220924D
:144D7000430390C020907B02209244038BC020907B02209249
:144D8400450386C020907B022092460381C020907B02209245
:144D980047037CC020907B022092480377C020907B02209241
:144DAC00490372C020907B0220924A036DC020907B0220923D
:144DC0004B0368C020907B0230907F03321409F056C022245F
:144DD400332430922903209228032092870302EF0E940202D6
:144DE80020903C032092830328822BE430E000270E947B0380
:144DFC000E94B40320903D0320928303288220E530E000273C
:144E10000E947B030E94B40320903E032092830328822EE430
:144E240030E000270E947B030E94B40320903F0320928303A0
:144E3800288222E430E000270E947B030E94B4032090400313
:144E4C002092830328822FE430E000270E947B030E94B403AD
:144E60002090410320928303288227E330E000270E947B0307
:144E74000E94B4030E94FC1C0BC003EF0E9402022224332417
:144E880030922903209228032092870320907B0230907F03A0
:144E9C00322430927F030C949935A89520907903222009F452
:144EB0003EC00E949D3520907E03222049F122242092830351
:144EC40019C020908303209285038AE893E0E22DFF27E80F80
:144ED800F91F2080288220918303332700270E947B030E94EA
:144EEC00B403809183038F5F8093830380918303883118F382
:144F000002EF0E940202222420927E030C9499352224209227
:144F14007E03209287033324309229032092280303EF0E9416
:144F280002020C94993580912803909129038931E0E09E075B
:144F3C0091F422243324309229032092280320907B02309087
:144F50007F03322430927F0381E0809379030C9499358091C2
:144F64002803909129038931E0E09E0710F00C949935209084
:144F78007B0230907F03322430927F038AE893E0E09128034B
:144F8C00F09129033197E80FF91F2082809128039091290362
:144FA000019690932903809328030C949935A89580912803F2
:144FB40090912903019690932903809328038130E0E09E0762
:144FC80091F08230E0E09E0791F08330E0E09E07B1F084304F
:144FDC00E0E09E0709F457C08530E0E09E0791F052C02090EB
:144FF0007B022092B70220907B022092B80222242092F00440
:1450040046C020907B022092B60241C020907B0230907F038B
:14501800321481F52090B7022092F2042090B8022092F104A6
:14502C002090B60228822FE130E000270E947B030E94B4039E
:145040002224332430922903209228032092870302EF0E9425
:1450540002022090E3032220D1F02090F30428822091F404B1
:145068000091A5021091A6020E940C0801E00E9472080BC035
:14507C0003EF0E94020222243324309229032092280320926E
:14509000870320907B0230907F03322430927F030C9499350B
:1450A400A8958091280390912903019690932903809328030E
:1450B8008130E0E09E0791F08230E0E09E0799F08330E0E03A
:1450CC009E07A1F08430E0E09E0709F453C08530E0E09E0757
:1450E00081F04EC020907B022092B90249C020907B022092BB
:1450F400BA0244C020907B022092BB023FC020907B02309060
:145108007F03321471F52090B9022092F5042090BA02209231
:14511C00F4042090BB022092F3040E9427060093F604809104
:14513000F50499278053984F9093A6028093A50222243324D6
:145144003092290320922803209287032FE130E000270E9467
:145158009403013011F40E94810602EF0E9402020BC003EFF9
:14516C000E94020222243324309229032092280320928703E5
:1451800020907B0230907F03322430927F030C949935809193
:14519400280390912903019690932903809328038130E0E0FA
:1451A8009E0771F08230E0E09E0779F08330E0E09E0709F458
:1451BC00F8C08430E0E09E0759F0F3C020907B0220928303AD
:1451D000EEC020907B0220928503E9C020907B0230907F039E
:1451E400321409F0D7C02090830328822AE230E000270E941C
:1451F8007B030E94B4032090850328822BE230E000270E9404
:14520C007B030E94B403209083033324322C222430921B03A6
:1452200020921A0320908503332440901A0350901B03420CE3
:14523400531C50921B0340921A0322243092290320922803F7
:145248002092870302EF0E94020220901A0330901B0344246C
:14525C0055243092C1022092C0025092C3024092C2024090BF
:14527000C2025090C3022090C0023090C10284E690E0A0E072
:14528400B0E05A924A923A922A928C019D010E94803D86E046
:1452980090E0A0E0B0E03A932A931A930A938C019D010E94E1
:1452AC00803D1801290180E092E0A0E0B0E0280E391E4A1E17
:1452C0005B1E8AE090E08A93810192010E94323E1093C102DD
:1452D4000093C0023093C3022093C20280EE98ECA0E1B0E06F
:1452E8003A932A931A930A938C019D010E94E73C1093D10278
:1452FC000093D0023093D3022093D202180130921903209271
:1453100018034090C2025090C3022090C0023090C10280E1DF
:145324009DECAEE0B0E05A924A923A922A928C019D010E94B1
:14533800E73C1093D1020093D0023093D3022093D20218012B
:14534C0030921703209216034090C2025090C3022090C002FB
:145360003090C10288EA97E0AFE0B0E05A924A923A922A925E
:145374008C019D010E94E73C1093D1020093D0023093D302C2
:145388002093D202180130921503209214030BC003EF0E946F
:14539C000202222433243092290320922803209287032090A5
:1453B0007B0230907F03322430927F030C94993580917B0294
:1453C400813F69F430907F03382630927F0381E080938803D5
:1453D8002224209289030C94993520908203222011F40C94B3
:1453EC00EE3380917B02823F51F422243324309229032092BB
:145400002803209282030C9499350E949D3520907E032220E1
:1454140011F40C94E033222420927E03A0908203BB24C501F9
:14542800843CE0E09E0709F4E5C2853CE0E09E0709F4EAC2D8
:14543C00863CE0E09E0709F488C3873CE0E09E0709F48FC376
:145450008A3CE0E09E0709F48CC48C3CE0E09E0709F449C598
:145464008F3CE0E09E0709F45AC68FEC8A159B0544F1C50132
:14547800803AE0E09E0709F45AC0813AE0E09E0709F4EDC020
:14548C00823AE0E09E0709F400C1843AE0E09E0709F413C139
:1454A000803AE0E09E0714F40C949935C501883BE0E09E0775
:1454B40009F473C1893BE0E09E0709F4CFC10C949935C501C9
:1454C800853EE0E09E0709F46CC7873EE0E09E0709F49DC7ED
:1454DC00893EE0E09E0709F4E4C78A3EE0E09E0711F40C9416
:1454F000C4328AEE90E08A159B0544F0C501853DE0E09E076A
:1455040009F42DC70C949935C5018A3FE0E09E0711F40C949B
:14551800CF328B3FE0E09E0711F40C94D7328C3FE0E09E0771
:14552C0011F40C94D6330C9499350091F404005D0E940202C3
:145540000FE20E9402020091F304005D0E9402020FE20E94A2
:1455540002020091F504005D0E94020200E20E94020200E248
:145568000E9402021AE00091F2040E945A3D00938303005D59
:14557C000E940202209083038AE0829D2090F2043324201881
:14559000310830921F0320921E03022D005D1F4F0E94020277
:1455A4000AE30E9402021AE00091F1040E945A3D009383038E
:1455B800005D0E940202209083038AE0829D2090F104332421
:1455CC002018310830921F0320921E03022D005D1F4F0E9407
:1455E00002020AE30E9402021AE00091F0040E945A3D0093D5
:1455F4008303005D0E940202209083038AE0829D2090F004B7
:1456080033242018310830921F0320921E03022D005D1F4F15
:14561C000E9402020AE00E9402020091F4040E940202009184
:14563000F3040E9402020091F5040E9402020091F2040E9470
:1456440002020091F1040E9402020091F0040E94020202EF06
:145658000E9402022224209282030C94993502EF0E94020216
:14566C0081E08093E5032224332430922B0320922A0380934F
:14568000A90289E790E090932D0380932C03209282030C941F
:14569400993502EF0E94020222242092E503332430922B0376
:1456A80020922A0381E08093A90280E19EE090932D038093AB
:1456BC002C03209282030C94993502EF0E940202A8952AE226
:1456D00030E000270E949403009365032BE230E000270E9475
:1456E400940300935D032224332430921D0320921C0313C005
:1456F8008EEE93E0E0911C03F0911D03E80FF91F8FEF8083EE
:14570C0080911C0390911D03019690931D0380931C038091FB
:145720001C0390911D038030E1E09E0728F322242092830366
:1457340015C0A8958EEE93E0998388832091830300270E9439
:1457480056030E94B4030E94B4030E94B403809183038F5F64
:14575C0080938303809183038D3038F32090650328822AE253
:1457700030E000270E947B030E94B40320905D0328822BE2AE
:1457840030E000270E947B030E94B4030C94000022242092C9
:1457980082030C94993502EF0E940202A89500EF0E940202A1
:1457AC008091F6048A5F8093830337C017E0009183030E94B5
:1457C000583D0093650322242092680323C02090650385E082
:1457D400829D900120563F4F209068033324220D331D0027F5
:1457E8000E949403202E332430921F0320921E0340907F03C6
:1457FC0055244224532440927F030E940202809168038F5FDF
:1458100080936803809168038530C8F28091830381508093A0
:1458240083038091F604815020908303821508F4C1CF81EF45
:1458380090E020907F0333242826392620927F0301EF0E94F0
:14584C00020200917F030E9402022224209282030C949935A0
:1458600002EF0E940202A89520E630E000270E949403202E9C
:14587400332430921D0320921C0303E611E00E9406020AE0A8
:145888000E94020280911C0390911D030996809383039CC061
:14589C001AE0009183030E94583D0093650322242092680352
:1458B00029C02090650386E0829D90012F593F4F209068039C
:1458C4003324220D331D00270E949403202E332430921F0311
:1458D80020921E0340907F0355244224532440927F03CE011E
:1458EC000296E0916803FF27E80FF91F2082809168038F5FF3
:145900008093680380916803863098F280911E0390911F03E4
:14591400807690708030890709F055C02C8028822B810A81AE
:145928000E940C1700E611E00E940602222428822E810D81F8
:14593C000E945C1700E611E00E94060280911E0390911F034C
:145950008F7190705C018130E0E09E07B1F08230E0E09E0718
:14596400B9F08430E0E09E07C1F08830E0E09E07C9F0813035
:14597800E0E09E07FCF0C5018031E0E09E07A9F019C005E592
:14598C0011E00E94060218C00AE411E00E94060213C00EE347
:1459A00011E00E9406020EC003E311E00E94060209C00CE252
:1459B40011E00E94060204C008E211E00E9406020AE00E946F
:1459C80002028091830381508093830320901C0330901D0317
:1459DC004090830355242414350408F459CFA89504EF0E9481
:1459F00002022224209282030C94993502EF0E9402020E947B
:145A0400FD152224209282030C94993502EF0E94020205E015
:145A18000E9455021801442437FC4094552447FC5094309297
:145A2C00D1022092D0025092D3024092D20220901A03309025
:145A40001B03442455243092CD022092CC025092CF024092BD
:145A5400CE024090CE025090CF022090CC023090CD02809000
:145A6800D2029090D3026090D0027090D1025A924A923A9238
:145A7C002A92830194010E94803D1093D1020093D002309344
:145A9000D3022093D20285E593E0A0E0B0E018012901280E40
:145AA400391E4A1E5B1E3092D1022092D0025092D302409214
:145AB800D2028BEA96E0A0E0B0E0BA93AA939A938A938101B5
:145ACC0092010E94E73C1093D1020093D0023093D302209348
:145AE000D20288E090E08A930E94323E0093830300EF0E942D
:145AF40002022090830330907F03322430927F03022D0E94B7
:145B080002024090D2025090D3022090D0023090D102209265
:145B1C00830330907F03322430927F03022D0E94020281EFCE
:145B300090E020907F0333242826392620927F0301EF0E94F5
:145B4400020200917F030E940202222420928203EEC702EF6D
:145B58000E940202F8940E946D2181E085BF82E085BF0C94EC
:145B6C00003E02EF0E94020200EF0E940202A89581E090E0AD
:145B800090931F0380931E03E3C080911E0390911F038130CF
:145B9400E0E09E070CF4C7C089E190E020901E0330901F0384
:145BA800821593050CF4BDC0910102E010E00E94703DF80191
:145BBC0086E091E0E80FF91F05901490F00109942FE230E007
:145BD00000270E94940300938303A7C020E330E000270E9405
:145BE4009403009383039FC021E330E000270E949403009397
:145BF800830397C022E330E000270E949403009383038FC0DF
:145C0C0024E330E000270E9494030093830387C025E330E095
:145C200000270E949403009383037FC02DE230E000270E94D0
:145C340094030093830377C02EE230E000270E949403009362
:145C480083036FC025E430E000270E9494030093830367C0DA
:145C5C0026E430E000270E949403009383035FC02DE330E062
:145C700000270E9494030093830357C02EE330E000270E94A6
:145C84009403009383034FC021E430E000270E949403009345
:145C9800830347C029E430E000270E949403009383033FC0D6
:145CAC002AE430E000270E9494030093830337C022E530E03F
:145CC00000270E949403009383032FC023E530E000270E9487
:145CD40094030093830327C024E530E000270E949403009319
:145CE80083031FC025E530E000270E9494030093830317C0D9
:145CFC0022242092830313C02224209283030FC022242092FE
:145D100083030BC022242092830307C022242092830303C0A8
:145D240081EF809383032090830330907F03322430927F0350
:145D3800022D0E94020280911E0390911F03019690931F0331
:145D4C0080931E0380911E0390911F038A31E0E09E0708F47E
:145D600014CF00917F030E940202222420928203E0C602EF7F
:145D74000E94020200EF0E940202A89581E090E090931F038D
:145D880080931E03A3C080911E0390911F038130E0E09E07E5
:145D9C000CF487C081E190E020901E0330901F0382159305F8
:145DB0000CF47DC0910102E010E00E94703DF80188E391E01A
:145DC400E80FF91F05901490F00109942224209283036BC04C
:145DD80027E330E000270E9494030093830363C023E330E0EB
:145DEC0000270E949403009383035BC029E330E000270E942A
:145E000094030093830353C02AE330E000270E9494030093BB
:145E140083034BC0209056032092830346C0209055032092E8
:145E2800830341C020907103209283033CC02090A70320927B
:145E3C00830337C028E430E000270E949403009383032FC051
:145E50002BE430E000270E9494030093830327C02DE430E09E
:145E640000270E949403009383031FC021E530E000270E94F3
:145E780094030093830317C021E430E000270E949403009387
:145E8C0083030FC02CE430E000270E9494030093830307C04D
:145EA00022242092830303C081EF80938303209083033090AE
:145EB4007F03322430927F03022D0E94020280911E03909196
:145EC8001F03019690931F0380931E0380911E0390911F031F
:145EDC008231E0E09E0708F454CF00917F030E94020222247C
:145EF000209282031EC60E94313B0E94833B05E00E94550237
:145F04001801442437FC4094552447FC50943092D10220921A
:145F1800D0025092D3024092D20220901A0330901B03442433
:145F2C0055243092CD022092CC025092CF024092CE024090B2
:145F4000CE025090CF022090CC023090CD028090D2029090BB
:145F5400D3026090D0027090D1025A924A923A922A928301FB
:145F680094010E94803D1093D1020093D0023093D30220930B
:145F7C00D20285E593E0A0E0B0E018012901280E391E4A1E18
:145F90005B1E3092D1022092D0025092D3024092D2028BEA99
:145FA40096E0A0E0B0E0BA93AA939A938A93810192010E94D8
:145FB800E73C1093D1020093D0023093D3022093D20202EFC7
:145FCC000E9402020E94B40300EF0E940202222420928303AF
:145FE00014C020918303332700270E9494030093650330902D
:145FF4007F03302630927F030E940202809183038F5F80933F
:14600800830380918303883540F388E090E04090D20250901B
:14601C00D3022090D0023090D1028A93810192010E94323E42
:146030000093830330907F03302630927F030E9402024090F1
:14604400D2025090D3022090D0023090D102209283033090B2
:146058007F03322430927F03022D0E9402020091F5040E9417
:14606C0002022090F50430907F03322430927F030091F4040E
:146080000E9402022090F40430907F03322430927F03009151
:14609400F3040E9402022090F30430907F03322430927F03D8
:1460A8000091F2040E9402022090F20430907F0332243092B7
:1460BC007F030091F1040E9402022090F10430907F033224E5
:1460D00030927F0383E080938303382630927F03082F0E9401
:1460E400020283E28093830330907F03382630927F03082F8B
:1460F8000E94020201EF0E94020281EF90E020907F033324EF
:14610C002826392620927F03022D0E9402022224209282034C
:1461200008C502EF0E94020200EF0E94020281E090E090937E
:146134001F0380931E0302C180911E0390911F038130E0E058
:146148009E070CF4E6C08BE190E020901E0330901F038215D2
:14615C0093050CF4DCC0910102E010E00E94703DF8018AE5E0
:1461700091E0E80FF91F05901490F00109942090AE032092C1
:146184008303C9C02090AF0320928303C4C02090AD032092C8
:146198008303BFC08091CE03873C20F481E090E05C0102C045
:1461AC00AA24BB24A0928303B2C02090CE0320928303ADC0E2
:1461C0002090640320928303A8C02090D60320928303A3C0F0
:1461D4002090AC03209283039EC02090AB032092830399C0D3
:1461E80020906E032092830394C020906F03209283038FC04D
:1461FC002090F304209283038AC02090F4042092830385C041
:146210002090F5042092830380C02090F204209283037BC040
:146224002090F1042092830376C02090F0042092830371C046
:146238004090C6025090C7022090C4023090C50220928303DC
:14624C0066C088E090E04090C6025090C7022090C4023090C9
:14626000C5028A93810192010E94323E1093D1020093D00244
:146274003093D3022093D20218012901209283034AC088E00A
:1462880090E04090D2025090D3022090D0023090D1028A9307
:14629C00810192010E94323E0093830338C083E080938303BA
:1462B00034C083E28093830330C02090E303222021F082E0AD
:1462C4008093830328C02AE330E000270E94940300938303AF
:1462D80020C02AE330E000270E949403002341F02090CF037F
:1462EC00222021F481E090E05C0102C0AA24BB24A0928303F2
:146300000CC02090C7032092830307C022242092830303C003
:1463140081EF809383032090830330907F03322430927F035A
:14632800022D0E94020280911E0390911F03019690931F033B
:14633C0080931E0380911E0390911F038C31E0E09E0708F486
:14635000F5CE00917F030E940202222420928203E8C302EFA4
:146364000E94020200EF0E9402022090AF0330907F033224F0
:1463780030927F03022D0E94020281EF90E020907F0333248F
:14638C002826392620927F0301EF0E94020200917F030E94D1
:1463A0000202222420928203C4C302EF0E94020200EF0E94B9
:1463B40002022AE230E000270E9494030093830330907F03FA
:1463C800302630927F030E9402022BE230E000270E94940304
:1463DC000093830330907F03302630927F030E94020281EFA2
:1463F00090E020907F0333242826392620927F0301EF0E942D
:14640400020200917F030E9402022224209282038EC302EF08
:146418000E94020200EF0E94020283E08093830330907F03F7
:14642C00382630927F03082F0E94020283E28093830330901F
:146440007F03382630927F03082F0E94020228E230E0002706
:146454000E9494030093830330907F03302630927F030E9464
:14646800020229E230E000270E9494030093830330907F0346
:14647C00302630927F030E94020281EF90E020907F03332463
:146490002826392620927F0301EF0E94020200917F030E94CC
:1464A400020222242092820342C302EF0E94020222242092CF
:1464B8008303288228E130E000270E947B030E94B4038CE07B
:1464CC0080938303282E288229E130E000270E947B030E9420
:1464E000B40380E09CE080938303282E28822AE130E000273A
:1464F4000E947B030E94B40380E09CE0A0E0B0E09093C90241
:146508008093C802B093CB02A093CA022224209283038FEF97
:14651C00809321018093220180932301809324018093250158
:1465300080E090E0A0E0B0E09093C5028093C402B093C702A8
:14654400A093C60228822BE130E000270E947B030E94B403E2
:146558002090830328822CE130E000270E947B030E94B40392
:14656C002090830328822DE130E000270E947B030E94B4037D
:14658000222420928203D5C202EF0E940202F89461E081E02E
:1465940085BF82E085BF0C94003E02EF0E940202E7D2222495
:1465A80020928203C2C202EF0E94020200EF0E940202009167
:1465BC00F5040E9402022090F50430907F03322430927F03A7
:1465D0000091F4040E9402022090F40430907F033224309286
:1465E4007F030091F3040E9402022090F30430907F033224B4
:1465F80030927F030091F2040E9402022090F20430907F0336
:14660C00322430927F030091F1040E9402022090F10430904F
:146620007F03322430927F032FE130E000270E949403009337
:1466340083030E9402022090830330907F03322430927F0314
:1466480088E090E04090C6025090C7022090C4023090C50228
:14665C008A93810192010E94323E1093D1020093D002309348
:14667000D3022093D202180130921D0320921C0388E090E016
:146684008A930E94323E009383030E9402022090830330901E
:146698007F03322430927F0320901C0330901D0320928303EB
:1466AC00022D0E9402022090830330907F03322430927F03F3
:1466C0004090C6025090C7022090C4023090C5022092830350
:1466D400022D0E9402022090830330907F03322430927F03CB
:1466E80088E090E04090CA025090CB022090C8023090C90278
:1466FC008A93810192010E94323E1093D1020093D0023093A8
:14671000D3022093D20288E090E08A930E94323E10931D034F
:1467240000931C0318012092830330907F03302630927F0382
:146738000E9402024090D2025090D3022090D0023090D10239
:14674C002092830330907F03322430927F03022D0E94020250
:146760004090CA025090CB022090C8023090C902209283039F
:1467740030907F03322430927F03022D0E94020281EF90E080
:1467880020907F0333242826392620927F0301EF0E940202FD
:14679C0000917F030E940202222420928203C3C102EF0E949C
:1467B000020281E080938603222420928203B9C103EF0E9449
:1467C4000202222420927E0333243092290320922803209270
:1467D8008203ABC180917B02803F59F481E0809389032224DC
:1467EC0020927F0320928703209282039CC180918903813047
:1468000009F090C120907B0220927F03222420928903A09025
:146814007B02BB24C501803BE0E09E0794F085ED8A159B05F9
:1468280024F102E010E095010E94703DF80182E390E0E80FCB
:14683C00F91F05901490F0010994C501803AE0E09E0709F487
:146850001DC1813AE0E09E0709F41CC1823AE0E09E0709F43E
:146864001BC1843AE0E09E0709F41AC160C1C501853EE0E0DF
:146878009E0709F44FC1863EE0E09E0709F4F0C0873EE0E0FF
:14688C009E0709F441C1893EE0E09E0709F430C18A3EE0E0B2
:1468A0009E0709F433C18D3EE0E09E0709F4C8C0853EE0E016
:1468B4009E070CF43CC1C5018A3FE0E09E0709F413C18B3F9F
:1468C800E0E09E0709F412C18C3FE0E09E0709F405C18D3FC8
:1468DC00E0E09E0709F4A4C08E3FE0E09E0709F4B3C021C15E
:1468F00080EB8093870380912001807F8093200181E08093B3
:14690400ED0383E08093EC038093EB0322243324309229039E
:14691800209228030AC181EB8093870380912001807F809376
:14692C00200184E08093ED0385E08093EC0383E08093EB0304
:14694000222433243092290320922803F2C082EB809387031F
:1469540080912001807F8093200189E08093ED0383E08093E8
:14696800EC038093EB03222433243092290320922803DBC028
:14697C0083EB8093870320907B0220927F0383E08093EC0336
:146990008093EB03222433243092290320922803C8C084EB93
:1469A4008093870320907B0220927F0385E08093EC0383E017
:1469B8008093EB03222433243092290320922803B4C085EB7E
:1469CC008093870320907B0220927F0383E08093EC03809341
:1469E000EB03222433243092290320922803A1C08BEC809362
:1469F400870322243324309229032092280397C08EEC8093B9
:146A080087032224332430922903209228038DC088EC8093B4
:146A1C00870322243324309229032092280383C08DEF8093A2
:146A3000870381E090E0909329038093280379C08DEE8093A3
:146A440087032224332430922903209228036FC08EEF80938D
:146A5800870322243324309229032092280365C086EE80938C
:146A6C0087032224332430922903209228035BC088EB809383
:146A8000820357C089EB8093820353C080EA809382034FC036
:146A940081EA809382034BC082EA8093820347C084EA809354
:146AA800820343C08FEC809382033FC08CEC809382033BC035
:146ABC0085ED8093820337C08AEC8093820333C087EC80933E
:146AD00082032FC084EC809382032BC085EC8093820327C05B
:146AE4008CEF8093820323C08AEF809382031FC08BEF80932B
:146AF80082031BC089EE8093820317C086EC8093820313C067
:146B0C008AEE809382030FC087EE809382030BC085EE809338
:146B2000820307C080917B028F3E19F402EF0E940202289658
:146B34000E94B03D0895222420927903209287033324309258
:146B480029032092280320907B0230907F03321439F481E0ED
:146B5C0080937E03222420927F0305C0222420927E03209227
:146B70007F03089500EF0E9402022224332430922903209220
:146B8400280319C0209128033091290300270E94940300933D
:146B9800830330907F03302630927F030E94020280912803A5
:146BAC00909129030196909329038093280380912803909107
:146BC00029038831E0E09E07F8F22224332430922903209250
:146BD400280381EF90E020907F0333242826392620927F0338
:146BE80001EF0E94020200917F030E94020208950E94C93D05
:146BFC00269700240B8211241D820C821A82098208822224BE
:146C1000209285032092A20320927E03A89580E09CE0A0E013
:146C2400B0E09093C1028093C002B093C302A093C2029AC3B5
:146C380020908503222009F0F4C100EF0E9402022224209293
:146C4C007F033324309229032092280332C020912803309101
:146C6000290300270E9494030093830330907F033026309221
:146C74007F03002319F00E94020216C085E190E02090280331
:146C8800309029038215930550F400E20E94020280E22090FF
:146C9C007F03282620927F0303C00B8003940B828091280332
:146CB000909129030196909329038093280380912803909102
:146CC40029038831E0E09E0730F2A090F404BB24C5018130D2
:146CD800E0E09E0709F438C08230E0E09E0709F43AC083308D
:146CEC00E0E09E0709F43CC08430E0E09E0709F43EC085306D
:146D0000E0E09E0709F440C08630E0E09E0709F442C087304C
:146D1400E0E09E0709F444C08830E0E09E0709F446C089302C
:146D2800E0E09E0709F448C08A30E0E09E0709F44AC08B300C
:146D3C00E0E09E0709F44CC08C30E0E09E0709F44EC053C096
:146D50008AE4E82E81E6A82E8EE6C82E4CC086E4E82E85E60D
:146D6400A82E82E6C82E45C08DE4E82E81E6A82E82E7C82EBF
:146D78003EC081E4E82E80E7A82E82E7C82E37C08DE4E82E74
:146D8C0081E6A82E89E7C82E30C08AE4E82E85E7A82E8EE626
:146DA000C82E29C08AE4E82E8CE6A82E89E7C82E22C081E487
:146DB400E82E85E7A82E87E6C82E1BC083E5E82E85E6A82E76
:146DC80080E7C82E14C08FE4E82E83E6A82E84E7C82E0DC090
:146DDC008EE4E82E8FE6A82E86E7C82E06C084E4E82E85E6BE
:146DF000A82E83E6C82E81E090E090931D0380931C0309C04B
:146E040080911C0390911D03019690931D0380931C038091EC
:146E18001C0390911D03883EE3E09E0778F30E2D0E9402028C
:146E2C0020907F032E2420927F030A2D0E94020220907F038B
:146E40002A2420927F030C2D0E94020220907F032C242092A9
:146E54007F030DE20E94020280E220907F03282620927F03FD
:146E68001AE00091F3040E945A3D802F805D80938303082FFF
:146E7C000E9402022090830330907F03322430927F031AE050
:146E90000091F3040E945A3D8AE0809F8091F3048019805D26
:146EA40080938303082F0E9402022090830330907F03322496
:146EB80030927F030DE20E94020280E220907F032826209259
:146ECC007F0314E60091F5040E945A3D84E6809F0091F50460
:146EE00000191AE00E945A3D802F805D80938303082F0E9454
:146EF40002022090830330907F03322430927F031AE00091E9
:146F0800F5040E945A3D8AE0809F8091F5048019805D809327
:146F1C008303082F0E9402022090830330907F03322430926E
:146F30007F0300E20E94020280E220907F03282620927F032D
:146F44001AE00091F2040E945A3D802F805D80938303082F23
:146F58000E9402022090830330907F03322430927F031AE073
:146F6C000091F2040E945A3D8AE0809F8091F2048019805D4B
:146F800080938303082F0E9402022090830330907F033224B9
:146F940030927F030BE30E9402028BE320907F032826209271
:146FA8007F031AE00091F1040E945A3D802F805D8093830375
:146FBC00082F0E9402022090830330907F03322430927F03D2
:146FD0001AE00091F1040E945A3D8AE0809F8091F1048019CC
:146FE400805D80938303082F0E9402022090830330907F03CE
:146FF800322430927F0300270E94020222242092830308C0D8
:14700C0000270E940202809183038F5F80938303209083034F
:147020000B80201498F3A8953CC180918503813009F037C19D
:147034002090A2032220E1F080E092E0A0E0B0E04090C2026A
:147048005090C3022090C0023090C102281A390A4A0A5B0A5C
:14705C003092C1022092C0025092C3024092C20222242092F2
:14707000A20303C02224209284034090C2025090C30220903C
:14708400C0023090C1028090CA029090CB026090C802709030
:14709800C902621873088408950880E092E0A0E0B0E068169B
:1470AC0079068A069B06F8F48090CA029090CB026090C802B1
:1470C0007090C902621873088408950881E090E0A0E0B0E0F2
:1470D400680E791E8A1E9B1E7092D1026092D0029092D302AA
:1470E8008092D20213013D822C8281E090E09A83898300EF44
:1470FC000E940202222420927F0380E09CE0A0E0B0E04090A4
:14711000C2025090C3022090C0023090C102281639064A0640
:147124005B0609F0B4C021E530E000270E949403013041F4AD
:1471380029E131E000270E9494030093830307C02FE230E0C7
:14714C0000270E94940300938303009183030E940202A895BC
:147160002090830330907F03322430927F0380E09CE0A0E0AD
:14717400B0E09093C1028093C002B093C302A093C20282E05B
:1471880090E09A83898381C088E090E04090C2025090C30208
:14719C002090C0023090C1028A93810192010E94323E109303
:1471B000D1020093D0023093D3022093D20288E090E08A937F
:1471C4000E94323E00937D032091C0023091C1020E94940362
:1471D8000093A4030C801D8009811A810016110629F50EEED4
:1471EC000E9402028EEE90E020907F03332428263926209215
:147200007F0381E090E0A0E0B0E04090C2025090C30220902E
:14721400C0023090C102280E391E4A1E5B1E3092C10220927C
:14722800C0025092C3024092C20237C08091A4038E3E19F4CB
:14723C0022242092A4030091A4030E9402022090A4033090AA
:147250007F03322430927F0381E090E0A0E0B0E04090C20299
:147264005090C3022090C0023090C102280E391E4A1E5B1E0E
:147278003092C1022092C0025092C3024092C20289819A81A7
:14728C0001969A83898380E092E009801A80801591050CF012
:1472A00077CF81EF90E020907F0333242826392620927F034A
:1472B40001EF0E94020200917F030E940202A8952224209242
:1472C8007B0281E090E090931D0380931C0341C081E080937A
:1472DC00830305C0809183038F5F80938303809183038436E4
:1472F000B8F3A89588E19CE920901C0330901D0382159305D6
:1473040020F40024039408822FC080917B02823F21F481E068
:147318008093850327C080917B02833F89F4809184038F5F8C
:14732C008093840381E08093A20382E0209084038215B0F4C6
:1473400000240394088212C080911C0390911D0301969093F7
:147354001D0380931C0380911C0390911D038034ECE99E0734
:1473680008F4B6CF4090CA025090CB022090C8023090C90242
:14737C008090C2029090C3026090C0027090C102261437045A
:147390004804590420F00880002009F44DCC26960E94BF3D18
:1473A40008950E94C23DA02E2197222420927C0320902601C3
:1473B800222009F01FC1AA2009F41CC18091AF03813009F095
:1473CC0017C1209025013090F504321401F185EF8093830301
:1473E000282E28822091C8023091C90200917D030E947B0361
:1473F4000E94B40305D12090F5042092250128822091C802B0
:147408003091C90200917D030E947B030E94B403F5D02090E5
:14741C0024013090F404321401F186EF80938303282E288239
:147430002091C8023091C90200917D030E947B030E94B403B7
:14744400DFD02090F4042092240128822091C8023091C90255
:1474580000917D030E947B030E94B403CFD020902301309063
:14746C00F304321401F187EF80938303282E28822091C80253
:147480003091C90200917D030E947B030E94B403B9D02090A9
:14749400F3042092230128822091C8023091C90200917D0355
:1474A8000E947B030E94B403A9D0209022013090F20432140F
:1474BC0001F188EF80938303282E28822091C8023091C902B3
:1474D00000917D030E947B030E94B40393D02090F204209263
:1474E400220128822091C8023091C90200917D030E947B038F
:1474F8000E94B40383D0209021013090F104321401F189EF9D
:14750C0080938303282E28822091C8023091C90200917D03BA
:147520000E947B030E94B4036DD02090F1042092210128827E
:147534002091C8023091C90200917D030E947B030E94B403B2
:147548005DD08A2D8F3F21F1A8822091C8023091C9020091A9
:14755C007D030E947B030E94B4034ED081E090E0A0E0B0E023
:147570004090C6025090C7022090C4023090C502280E391E3C
:147584004A1E5B1E3092C5022092C4025092C7024092C602CC
:1475980084EF9FEFA3E0B0E04090CA025090CB022090C80208
:1475AC003090C902281639064A065B0618F081E0809326016F
:1475C00000E40E94D91E2224332430921D0320921C0309C021
:1475D40080911C0390911D03019690931D0380931C03809115
:1475E8001C0390911D038032EEE49E0778F300E40E94ED1E0A
:1475FC0021960E94B03D089581E090E0A0E0B0E04090CA021B
:147610005090CB022090C8023090C902280E391E4A1E5B1E46
:147624003092C9022092C8025092CB024092CA0288E090E024
:147638008A93810192010E94323E1093D1020093D00230935C
:14764C00D3022093D20288E090E08A930E94323E00937D03B4
:14766000089521974090C6025090C7022090C4023090C50283
:147674002092830328822DE130E000270E947B030E94B40362
:1476880088E090E04090C6025090C7022090C4023090C502D8
:14769C008A93810192010E94323E1093D1020093D0023093F8
:1476B000D3022093D202180129012092830328822CE130E028
:1476C40000270E947B030E94B40388E090E04090D2025090B6
:1476D800D3022090D0023090D1028A93810192010E94323E70
:1476EC0000938303202E28822BE130E000270E947B030E9474
:14770000B4032196089521974090CA025090CB022090C802EF
:147714003090C9022092830328822AE130E000270E947B0392
:147728000E94B40388E090E04090CA025090CB022090C80259
:14773C003090C9028A93810192010E94323E1093D102009361
:14775000D0023093D3022093D202180129012092830328820F
:1477640029E130E000270E947B030E94B40388E090E04090AF
:14777800D2025090D3022090D0023090D1028A93810192012D
:14778C000E94323E00938303202E288228E130E000270E94E4
:1477A0007B030E94B403219608950E94C23D5801A89500EF84
:1477B40019E422E030E06BD005C0C501885E93405C0196D070
:1477C80087EE93E08A159B05B0F39DD0A89505C0C5018456D4
:1477DC0090405C0189D083E690E08A159B05B0F390D0A895BB
:1477F00004C0C5010A975C017DD089E090E08A159B05B8F3ED
:1478040084D0A89504C0C50101975C0171D0AA20D1F7BB20B2
:14781800C1F700E711E121E030E037D09698A89508E813E164
:14782C0020E030E030D0969AA89500E117E220E030E029D0E8
:147840009698A89508E813E120E030E022D0969AA89500E78F
:1478540011E121E030E01BD00E94B03D08950E94C23DA02E97
:147868002A2C209432B2322032BA00E516E420E030E00BD016
:14787C0022B22A2822BA00E516E420E030E003D00E94B03DA5
:1478900008950E94A83C249780E090E0A0E0B0E0FE01808324
:1478A4009183A283B38313C0A89581E090E0A0E0B0E0FE0171
:1478B8002080318042805380280E391E4A1E5B1EFE012082C7
:1478CC00318242825382FE012480358046805780FE01608088
:1478E0007180828093806214730484049504F4F2289608953F
:1478F400969800E516E420E030E0C9DF969A00E516E420E0AC
:1479080030E0C3DF089508EF14E221E030E0BDDF969808E864
:14791C0013E120E030E0B7DF969A08EF14E221E030E0B1DFFF
:14793000089517FF0895109501951F4F0895A02FB12FE22FED
:14794400F32F01900D920020E1F708953A932A931A930A9374
:1479580008956894DA92D12E04C0E894DA92D12ED32617FF5D
:14796C0004C0109500950F5F1F4F37FF04C0309520952F5F2B
:147980003F4F0E94CE3CD7FE04C0109500950F5F1F4FD990A1
:147994000895689401C0E894EA92FA928A93EE24FF2480E14E
:1479A800000F111FEE1CFF1CE216F30618F0E21AF30A0395DD
:1479BC008A95A1F716F40E2D1F2D8991F990E9900895E8943A
:1479D00001C068942FD0CC2408C0E89401C0689429D037FDC9
:1479E40053D0B7FD5AD0772488249924AA24BB2441D0C1F01B
:1479F80044D0B1F0E8E2000F111F221F331F771C881C991C3E
:147A0C00AA1CBB1C88169906AA06BB0628F0881A990AAA0A0A
:147A2000BB0A0395EA9559F726F4082D192D2A2D3B2D13C0FF
:147A34007A928A929A92AA92BA92CA92EA938A939A93AA9302
:147A4800BA938B859C85AD85BE85C32E0EF0CB260895C7FCF7
:147A5C0017D0B991A99199918991E991C990B990A9909990E9
:147A70008990799024960895E02FE12BE22BE32B0895E82F9F
:147A8400E92BEA2BEB2B089500951095209530950F5F1F4F82
:147A98002F4F3F4F089580959095A095B0958F5F9F4FAF4FA3
:147AAC00BF4F0895689401C0E8942A93FA92EA92FF24EE24E8
:147AC00020E1000FFF1CEE1CE11610F0E11A03952A95B9F784
:147AD4000EF40E2DE990F990299108950A921A928A939A9376
:147AE800029FC001129F900D039F900D8C0199918991199021
:147AFC00099008950E94CD3D7F920E94E63D39F177240E9457
:147B1000EC3D19F48C019D0120C0089FB02CA12C289F902C4D
:147B2400812C189FA00C911C871C099FA00C911C871C199F91
:147B3800900C811C0A9F900C811C389F800C299F800C1A9FAE
:147B4C00800C0B9F800C0B2D1A2D292D382D7F900C94DB3D62
:147B6000E4E0A990B990E2FD0895C990D990E3FD0895E99097
:147B7400F9900895E8E00C94B13DEE270C94B13DBA92AA9256
:147B88000895DA92CA920C94C23DFA92EA920C94C53D8A921F
:147B9C009A92AA92BA92EA938A939A93AA93BA9389859A85A3
:147BB000AB85BC850895B991A99199918991E991B990A990EF
:147BC4009990899024960895EE27E02BE12BE22BE32B089530
:147BD800EE27E82BE92BEA2BEB2B0895FA93EA93BA93AA9301
:147BEC009A938A933A932A931A930A939A928A927A926A9217
:147C00005A924A923A922A921A920A920FB60A920895099041
:147C14000FBE099019902990399049905990699079908990EE
:147C28009990099119912991399189919991A991B991E99115
:147C3C00F99108950F920990002031F0000F111F221F331FC0
:147C50000A94F8CF0F900895112319F0000F1A95FBCF08951D
:147C64000F920990002031F036952795179507950A94F8CF5D
:147C78000F9008950A921A92002411240030010741F0169507
:147C8C00079510F4020E131E220F331FF5CF002D112D1990A8
:147CA00009900895AA93BA93EA93FA930A92AF81B885ED818F
:147CB400FE810030010731F0C8950D92319601501040F7CFBA
:147CC8000990F991E991B991A99124960895AA93BA93EA9329
:147CDC00FA930A92AF81B885ED81FE810030010729F001902F
:147CF0000D9201501040F8CF0990F991E991B991A99124969E
:147D040008950E94C23DA02E2090EE043090EF04222011F4C3
:147D1800332029F08A2D8A3011F40DE0F0DF5D9BFECFACB890
:147D2C000A2D11270E94B03D08950E94A83C0E94C93D622EEA
:147D4000732EA297ECA4FDA4862D972D8030E0E09E074CF458
:147D5400CC24C394809590958F5F9F4F682E792E01C0CC24D0
:147D6800222429A28C2F9D2F8196A82EB92E8A2D9B2D019784
:147D7C00282E392EA82EB92E2E2D3F2D062D172D0E94AD3CB0
:147D9000E02FF12F84E592E0E80FF91F4080E22DF32D408215
:147DA4002E2D3F2D062D172D0E94B13C602E712E6620F9F65C
:147DB8007720E9F6CC2059F08A2D9B2D0197282E392EA82E62
:147DCC00B92E8DE2E22DF32D80832A2D3B2D08A519A50E944F
:147DE0009F3CA2960E94BF3D2496089510937A02009379025A
:147DF40008952091790230917A020DE61EE40E943E3E802FB3
:147E0800912F875C9F4C9F7790937A0280937902082F192F16
:027E1C000895C7
:00000001FF
